:020000040800F2
:10500000F81B0020D5500008CD8800080580000856
:105010000000000000000000000000000000000090
:1050200000000000000000000000000041970008A0
:105030000000000000000000A99000087D98000812
:10504000E7500008E7500008E7500008E750000864
:10505000E7500008D95C0008E7500008E750000856
:1050600000000000E7500008015C0008E75000085D
:10507000E75000082D85000800000000E7500008F8
:1050800000000000E75000080000000000000000E1
:10509000E750000800000000E7500008E750000853
:1050A000E7500008E7500008E750000865A1000835
:1050B000E7500008E7500008000000000000000072
:1050C0000348854600F0E8FC00480047D9B40008D2
:1050D000F81B00200448804704480047FEE7FEE72D
:1050E000FEE7FEE7FEE7FEE719990008C150000859
:1050F00030B50B46014600202022012409E00D4670
:10510000D5409D4205D31D469540491B25469540F7
:1051100040191546521E002DF1DC30BDF0B51FB40C
:105120000646002082B005464024019100901BE015
:10513000019922460F46304600F098FB049A059BE1
:10514000801A994110D310461946224600F07EFB82
:10515000361A8F410197224601200021009F00F05E
:1051600075FB38184D4100902046641E0028DFDC96
:10517000019B00982946324607B0F0BD03460B4319
:105180009B0703D009E008C9121F08C0042AFAD2FD
:1051900003E00B780370401C491C521EF9D2704783
:1051A000D2B201E00270401C491EFBD270470022BF
:1051B000F6E710B513460A4604461946FFF7F0FF16
:1051C000204610BD30B504460020034600E05B1CBD
:1051D000934203D2E05CCD5C401BF8D030BDF8B503
:1051E00002464A40D40F42004B0052085B089A42E4
:1051F00002D20246084611464A0023D0C30D4A0097
:10520000DDB2120EAD1A202D35DA49020126490A07
:10521000F6058A19002C00D0524220214F1B11465E
:10522000B9402A411018C20D9A4221D0002C17D043
:10523000012D08DCDA05801AD20F8019D207DBB203
:1052400000F040FBF8BDDA05801A012340001B0680
:10525000C01880185A428018CA0F1043490007E04E
:105260004908C2071143DA05801A801940088018DE
:1052700000F020FBF8BD61000122511A001BF7E786
:105280000122D2075140AAE70122D2075040A6E7E7
:1052900070B502464A40D50F40004A00ED0740086D
:1052A0005208002814D0002A12D0C40DD30D410298
:1052B0000120C0055202490A520AE41A09181218BC
:1052C0007D34914201D3641C00E04900002C01DAD6
:1052D000002070BD0023914201D3891A0343400886
:1052E00049000028F7D100290AD0914202D10121BA
:1052F000C90705E0914201D2012101E00121C94322
:10530000E005C018401900F0D5FA70BD420005D084
:105310004200120E52428A4201DB00207047C9054A
:1053200008187047F0B507460846584087B0C00FC8
:10533000049048000E46590040084908BC1A8841AC
:1053400005D2384631461E4617460B4602465800DF
:10535000400810434CD0300D039040055900400DDB
:10536000490D0590401A0290402872DA1803012175
:10537000000B09050843019004980092002805D00D
:1053800001995242002088410092019002984021E8
:105390000A1A0199009800F059FA05460C466B4626
:1053A00007CB00F074FAC0197141039A0E0D002367
:1053B000D71756401A467A40164344D0049A002A1A
:1053C0002DD0029A012A039A15DC1205C01A9141C8
:1053D00001263605001C7141D20F059ED2070093AD
:1053E000019202962A46234600F0B2FA07B0F0BDB9
:1053F00038463146FAE71605224A0F46B218C01A57
:10540000B74101210905001C4F4100187F41114699
:1054100018187941E20F10436D19644113E0E20757
:105420006D0815436408C2071443039A0126120548
:10543000C01A91413605001C7141CE074008304327
:105440004908C01851412A46234600F074FACDE7B6
:10545000FFE7049801224000C117121A00238B4174
:1054600004983146C417381AA141EEE730B401243C
:10547000E407634030BC55E730B40124E4076140E1
:1054800030BC4FE70000E0FFF0B51FB488B00B99C7
:105490000998002448400999C00F4900490809911A
:1054A000C0070B990090490049080B910999089889
:1054B000A64608431CD00B990A98084318D00998AF
:1054C00001244000420D4800410D099824050003C5
:1054D000000B204309900B980003000B20430B9016
:1054E00050181C494018002201901446104605E04F
:1054F000002001460DB0F0BD032801DA034600E0AC
:1055000003239C46C11A0AAE0AE05F0008ADED5BBA
:105510004F00F75B7D430027AA187C41491C5B1EA6
:105520006145F2DD410004AB5A522104120C0A43DA
:10553000240C401C0828DFDB01980290009970467B
:1055400001910090059B049A0799069800F000FAD3
:10555000D0E700000DFCFFFFF0B50C465C4085B0C5
:10556000E40FE40703944C000026640859009446B5
:10557000490802460296224321D062460A431ED0C1
:105580006200570D4A000E032303550D0124024605
:105590002C492405781B1B0B360B4018234326434C
:1055A000614600901C46501AB44103D30098401C39
:1055B000009002E0921800985B41002803DA002076
:1055C000014605B0F0BD00200121090507468646C9
:1055D00011E064461D46141BB54106D36546521BB7
:1055E000B341744607430C43A646CD07400849081B
:1055F000284392185B4105460D43EAD110461843F3
:1056000013D06046194650407140084306D06046AA
:10561000101AB34106D20122002306E00022012322
:10562000DB0702E00122D2435310009874460105C3
:10563000381C6141029C039D0019694100F07BF90F
:10564000BFE70000FD03000070B54B005B0803439B
:105650000BD04B005C0D002633466542B341D41796
:10566000AD1AA34102DB0020014670BD12053018BF
:10567000514170BDC217C10F504010B54018CA0744
:105680009623002100F01EF910BD10B500229623CC
:10569000114600F017F910BD0EB5C217C10F5040EA
:1056A000CA0740180021054B0293019200910A4657
:1056B0000B4600F04DF903B000BD000033040000BC
:1056C0000EB505490291002100910A460B46019151
:1056D00000F03EF903B000BD330400004100400279
:1056E0000122400AD205090E80187F2901DA002024
:1056F0007047962903DC9622511AC84070479639A4
:105700008840704770B5CD0F4A0009030123090B8B
:105710001B0519430B4BED070024520D9A4201DA89
:10572000002070BD074B34339A4203DC9A1A00F014
:105730009DF802E00449511888402C43F1D04042C2
:1057400070BD0000FF030000CDFBFFFF4A0009030E
:105750000123090B1B051943094B10B5520D9A4241
:1057600001DA002010BD064B34339A4203DC9A1A4A
:1057700000F07CF810BD03495118884010BD0000AE
:10578000FF030000CDFBFFFFC20FD207400040081F
:105790000BD0C10D0723DB01C91840020905400ADF
:1057A0001143C2084007114370470020014670476B
:1057B00010B5002904DB0124E40740428C41214656
:1057C000002B04DB1C460123DB075242A3418B4222
:1057D00000D1824210BD000010B5002904DB012475
:1057E000E40740428C412146002B04DB1C46012388
:1057F000DB075242A341994200D1904210BD000004
:10580000CB0FDB07490010B5490802460A4307D011
:105810000A0D07240903E401090B121B002A01DC0D
:10582000002010BDC900440F0C43C100E018D20590
:10583000801800F03FF810BD0122D207002800DBDD
:10584000101A002900DB511A8142704710B5202A36
:1058500004DB0146203A9140002010BD91402023F6
:105860009C1A0346E3401943904010BD10B5202A0E
:1058700004DB0846203AD040002110BD0B46D3403F
:10588000D0402024A21A91400843194610BD10B5FB
:10589000202A06DBCB170846203A1041C1170B43DC
:1058A00006E00B461341D0402024A21A9140084341
:1058B000194610BD002904DA401C490001D14008F6
:1058C0004000704770B40024050C05D1102400047A
:1058D00002D1002921D01124050E01D10002083483
:1058E000050F01D10001241D850F01D18000A41CEA
:1058F000002801DB4000641C002908D020252E1B55
:105900000D46F540A14000D001212943084301067E
:105910001B1B000ADB1D02D5002070BC7047DB0595
:10592000181880180029F8DA401C4900F5D170BC1D
:1059300040084000704710B5002B08DA0024401CD6
:10594000614192185B411A4301D14008400010BDEB
:10595000F0B51FB482B005460C0003D0084604F031
:10596000B5FC02E004F0B2FC203002460090214673
:105970002846FFF76BFF049B059A04460F46184321
:105980001143084314D0184610431BD000984021FF
:105990000A1A18460599FFF769FF05460E46009A50
:1059A00005990498FFF752FF084305D0012004E051
:1059B0002046394607B0F0BD0020C11705430E430D
:1059C0002C43374300990E986305401A7905E40A81
:1059D00000220C43FD0A0A3002D500200146E9E707
:1059E0000105101969410C9C0D9D00196941FFF7D3
:1059F000A2FFDFE7FEB500231A461B1A8A4103DB2C
:105A00000020014603B0F0BD4A000D0301212D0B1B
:105A10000905520D0D43D10702D100186D41521EE8
:105A20005110FF31FF310131002704463E46384610
:105A3000009701910246012100200905FFF716FF9A
:105A4000C3197141F818324684468E464A41614670
:105A50002846611A904104D36046241A954176463F
:105A60001F46241900986D41401C00903428E1DD48
:105A7000F91930467041091BA84103D20022D243D4
:105A8000134601E00022134601980105381C7141BC
:105A9000FFF751FFB6E70000064C0125064E05E072
:105AA000E36807CC2B430C3C98471034B442F7D33F
:105AB000FFF70AFBC8C30008E8C3000870B58C18DC
:105AC0000578401C6B075B0F01D10378401C2A113D
:105AD00006D10278401C03E006780E70401C491C79
:105AE0005B1EF9D12B0705D40023521E0DD40B7079
:105AF000491CFAE70378401CCB1A921C03E01D787E
:105B00000D70491C5B1C521EF9D5A142D8D3002050
:105B100070BD000038B50446064805490068FFF727
:105B2000E7FA604300E0401E00900028FBD138BD3A
:105B300040420F0084010020F8B5044600688168E7
:105B40008907890F012902D10168C90722D181681B
:105B5000114A10261140012500290ED181682943E0
:105B600081600120FFF7D6FF01F026F807460CE020
:105B700001F022F8C01B0A2807D9606D3043606528
:105B8000A06D2843A0650120F8BD20680068C043CF
:105B9000C007EDD10020F8BD170000801FB50B48ED
:105BA00000900B4801900B4802900B480390694607
:105BB0000A4804F081FF0A4A08481146083904F0EF
:105BC00069FE00F06DFA002004B010BDD5C10008D8
:105BD000B1C1000811C200080FC2000890010020E6
:105BE0001000002010B500231A4603E0845CE3187F
:105BF0009BB2521C8A42F9D3D84380B210BD000038
:105C000010B5034800F094FD024800F091FD10BD6E
:105C1000981700205017002030B5446C1C252C40EC
:105C20000125A540046C6560046863608368102BDF
:105C3000036803D099600068C26030BD9A60006854
:105C4000C16030BD1449012048720A4602205E320C
:105C5000507203203C3A507204200E3A50720F48A2
:105C60000D4B0078087022310870203108770C49FC
:105C70005A1C0878587149789971233318715971F1
:105C8000203318775977107551751A461E321075E2
:105C90005175107651767047E81100203E010020C2
:105CA0006001002010B503F021FD202003F0DCFD91
:105CB000012005F06BF9002003F0D6FD044805F043
:105CC00009F8044805F0B8FA002005F0EDFA10BD17
:105CD0000001002083800000F8B503F0D3FD05200B
:105CE0000121000700F054FF0025134C002800D0CC
:105CF0006560124E0221304600F04AFF002814D1A0
:105D0000012020700E48808F00280DD001229702BC
:105D10003946304600F049FF0A2004F02BFD0022EE
:105D20003946304600F041FF6560012000F068FE12
:105D3000022000F065FEF8BD700100200004005054
:105D4000E80D00207047000010B5084900224A61A4
:105D500007494B684C1523434B604B680824234389
:105D60004B60C009C001026010BD0000E0170020B8
:105D7000002002407FB500250C460646039500F042
:105D80000FFEE009029003A901960095684600F015
:105D90009FFD002804D000F0D7FD002004B070BDA6
:105DA00000F0D2FD0120F9E710B5002302E0C45C49
:105DB000CC545B1C9342FAD310BD000010B5214AAD
:105DC00000219069C305204804D541690223194385
:105DD0004161911593699B0505D5436901242343CE
:105DE00043616302194393695B0505D54369082440
:105DF00023434361E301194393691B0505D54369B7
:105E00000424234343616302194393699B0405D52A
:105E100043691024234343616302194393699B033D
:105E200004D5446920231C43446119439369DB036F
:105E300005D54369402423434361A0020143916196
:105E400010BD000000200240E017002070B505469C
:105E500000F0B2FE0646184C0AE0681C08D0002D7F
:105E600004D000F0A9FE801BA84201D9032070BD18
:105E7000A069C007F1D1A069800701D50220A06107
:105E8000A069C00511D4A06980050ED4A0694005A1
:105E90000BD4A069000508D4A069800405D4A069CA
:105EA000800302D4A069C00303D5FFF787FF012058
:105EB00070BD002070BD000000200240F8B51746FC
:105EC000002605460C4600F06BFD09E0294602203D
:105ED000226800F047FD002804D1241D2D1D361D29
:105EE000BE42F3D300F030FDBE4201D20020F8BD27
:105EF0000120F8BD10B5084902460020054B49793C
:105F000005E044001C5B944203D0401CC0B28842B0
:105F1000F7D310BD8C1300207000002010B500F0E6
:105F20003CFE10BD10B5094801F05CF880B2FFF7E7
:105F3000C7FB074A074BFFF7A7FA0022064BFFF7FC
:105F40000BFBFFF703FC80B210BD0000041600201D
:105F5000F853E3A59B843E4000408F4070B5002479
:105F6000204603F039F847494748A200641CE4B2D0
:105F70008150142CF9D3464944480A7A0275497A6B
:105F8000417544490A780276497841763F490520AF
:105F9000133148720A2005F03FF97D20400105F0D9
:105FA00055F93A49002213310C2005F01FFA00215F
:105FB0000C2005F02DFA384801F014F8344C012576
:105FC000203C6085AD0309E0334801F00BF880B256
:105FD0006085218FFF392D39884206DB218F80B201
:105FE0008842F1D349198842EED8022005F064F9BD
:105FF000002002F0F1FF294D00210F2005F08CF860
:1060000028422064F8D0206C411C38D0400435D59B
:106010008122D20100210F2005F0BDF900211020BE
:1060200005F07AF841061948490E0022C73005F0FC
:10603000A9F8164DC735687A05281FD102221549DF
:10604000681DFFF7BFF8002818D11148AE7C6671B3
:106050000422691C3830FFF791F8294613310846AD
:1060600072000D466930FFF789F8607929464200D1
:1060700005484838FFF782F80320207070BD04F00F
:1060800099F90000FFFF0100EC13002049120020E5
:1060900090000020600100200416002000D027247A
:1060A00010B5144C1448224610321146083904F039
:1060B000F1FB0022114BE168A068FFF74DFA104A8E
:1060C000104B05F017FB00220F4BFFF7D5F900220C
:1060D0000E4BFFF7D9F9FFF793FB20600022134620
:1060E000E168A068FFF764FB01D0206810BD0020C4
:1060F000206010BD000000209001002000AA8F4009
:106100006C45D9CC955BC83F0000F03F40A5E54009
:1061100010B5084800F096FA0A21064800F032FA55
:10612000044800F01DF9800503D5024800F01AF973
:1061300080B210BDA8150020F8B52F4D0022012116
:10614000284600F032FDFFF7E3FFFFF79EFA2B4EE3
:106150003146FFF79DF82A4C0122A06011462846DF
:1061600000F023FD2749A068002588423EDB207807
:10617000254F002815D02570FFF7CAFFFFF785FAD5
:106180003146FFF785F8A060FFF7FEFA00223B4694
:10619000FFF76CF900221D4BFFF776F9FFF730FB94
:1061A0006060A068FFF7F0FA00223B46FFF75EF957
:1061B000174A184BFFF768F906460F466068FFF765
:1061C000E3FA134A144B5242FFF75EF932463B465C
:1061D000FFF7A8F8FFF714FB10496060884201DD63
:1061E000616004E0FF21C905C84200D365606068B2
:1061F000FFF774FAC0B2F8BD0004005000401B4421
:10620000480000200000604000000C4000E06440B6
:106210003333333333B33040CCCCEC3F0000C8428F
:10622000F8B5054604464035287C0026012808D0EC
:1062300001202874206881688907890F01290ED1FF
:1062400001E00220F8BD0168C90708D0606D202177
:10625000084360650126002028743046F8BD616D52
:10626000FF2201329143022211436165C16889070F
:10627000890F0091C16889088900C1602068816820
:1062800092071143816000F097FC07460EE000F092
:1062900093FCC01B0A2809D9606D02218843102194
:1062A00008436065002028740120F8BD20688068DC
:1062B0000028ECDB2068C168009A1143C160606D62
:1062C00080088000401C6065C5E70000F8B5064600
:1062D0000D464036317C01290DD001213174016811
:1062E0008A68520709D5416D20221143416500207B
:1062F00030740120F8BD0220F8BD174B6A68D8053C
:1063000047109A42154C8A6A2B6812D05B035B0BCC
:106310001A438A622968490305D5A1680143A1602F
:106320000A20FFF7F7FB2868800312D5A0683843DE
:106330000EE05B035B0B9A438A622968490302D52E
:10634000A1688143A1602868800302D5A068B84392
:10635000A06000203074F8BD01100000002701404B
:10636000406D70470068006C7047000070B5040015
:1063700006D0606D264600254036002802D006E093
:10638000012070BDA5653574204600F0D3F8606D1E
:10639000C00603D421688868400705D5606D1021C8
:1063A000084360653574EBE7606DFF22013290436E
:1063B00002221043606588688207920F5B48012AB9
:1063C00002D10A68D2072BD1032362689B079A4245
:1063D00005D05B429A4202D05B009A4209D10A6919
:1063E000920092080A6121680A6963681A430A6187
:1063F0000CE00A69920092080A6181680F229204F7
:106400009143816081686268114381602168CA6834
:1064100018239A43CA602168CA68A3681A43CA60ED
:10642000816801225206914381608168A28E5206E2
:106430001143816020688168C90004D48168012209
:106440001207114381602068C168394A1140C16058
:106450002069E168022825D0002001432046203031
:106460000278037B52035B001A431143226B1143F2
:10647000A26992031143E269D20311432268D368EF
:106480001943D160616A0A46FF3AC23A05D0A26A4E
:1064900011432268D3681943D16042780121012A4F
:1064A00002D00BE00420D8E70078002823D0606DEC
:1064B000202210436065A06D0843A065E06B0128B1
:1064C00020681FD00169C90703D001694908490044
:1064D000016120684169C908C900416120684169BA
:1064E000A26B11434161A565606D80088000401C6E
:1064F0006065002070BD2068C26801231B041A4338
:10650000C260DBE70269FF239B009A4302612068B7
:106510000269236CA66C1A43636C33431A4302610D
:10652000206802690A430261D3E7000000270140A6
:106530001902FEFF10B586B0044614216846FEF726
:1065400036FE0E492068884216D10D48416B42152F
:1065500011434163C16A01221143C162C06A6946A5
:10656000104005900220009003200190002002902E
:106570000520000700F050FA06B010BD00240140CD
:1065800000100240F8B504464069254640350E46E5
:1065900008280BD02068C068C00709D0606D202192
:1065A00008436065002028740120F8BD082700E03A
:1065B0000C2700F001FB009011E0701C0FD0002EA2
:1065C00005D000F0F9FA0099401AB04207D9606D81
:1065D000042108436065002028740320F8BD20686A
:1065E00000683842E9D0606D0121490208436065C6
:1065F0002068C16809058A0F0C21002A1BD12022BE
:10660000125D002A17D10268120714D58268530759
:106610000122002B08DB43688B434360606D13024B
:1066200098431043606506E0606D20231843606561
:10663000A06D1043A065A069002801D12068016009
:106640000020F8BD70B5044621680020896849071C
:1066500021D425464035297C01291CD001212974EB
:10666000E169012904D02046FFF766FA002811D11C
:10667000616D0A4A1140FF22013211436165002118
:10668000A165297422681C21116021688A6804238D
:106690001A438A6070BD022070BD0000FEF1FFFF4A
:1066A00030B5014620314A790023022A04D0042261
:1066B000C2630B71012030BD026814680E25AC4323
:1066C000146002681468640864001460446C1C223E
:1066D000144001221546006CA54045604A711846D9
:1066E0000B7130BD70B50024014620314A79022A71
:1066F00003D00421C163012418E0026813680E2549
:10670000AB431360026813685B085B001360436C63
:106710001C221340012215469D40036C5D604A71A6
:1067200000220A71816B002900D08847204670BD85
:10673000F0B4016C0D6801680C68466C1C230422DF
:106740001E401746B7402F420ED067070CD50C6885
:10675000A40602D40C6894430C60416C19408A4032
:10676000016C4A60016B1AE00227B74002462F40D5
:106770002032002F17D0A70715D50C68A40605D422
:106780000C680A25AC430C6001215171446C022154
:106790001C40036CA140596000211171C16A00299D
:1067A00018D0F0BC08470827B7402F4212D0240762
:1067B00010D50C680E25AC430C60446C01211C40C4
:1067C0000B46A340046C6360C163517100211171D9
:1067D000416BE4E7F0BC704770B504003CD01F4843
:1067E000256814212818FEF783FC800060641C488B
:1067F0002064022120462030024641712968194850
:10680000E3680140A068666918432369334318436D
:10681000A3691843E3691843236A184308432860AF
:106820000121A0688903884210D00D488030836A16
:10683000656C1C210D400F26AE40B3438362656C2E
:1068400063680D40816AAB400B4383620020E063C4
:1068500001215171107170BD012070BDF8FFFDBFA5
:10686000000002400F80FFFFF8B504468C46203040
:1068700001790025012909D00126067141790027F7
:10688000012905D0077102252846F8BD0220F8BD70
:1068900002214171E76320680168490849000160ED
:1068A00061462046FFF7B8F9206B00282068016890
:1068B00001D00E2205E004229143016020680168A6
:1068C0000A22114301602068016831430160DBE75F
:1068D000F8B51A4E0546307C0F46012807D0012036
:1068E00030741748FFF7B2FA010002D021E002200D
:1068F000F8BD0020C04338606C6814E02046FFF704
:1069000023FA0F48FFF7A2FA01460E48426808230F
:106910009A434260426843159A434260002901D07D
:106920003C6006E08034A8686A68C0018018A04214
:10693000E4D8002030740846F8BD0000E0170020BD
:1069400050C3000000200240054841680222114364
:1069500041604168012211434160002070470000FE
:1069600000200240F8B50C4C1646207C0F4601284A
:1069700008D0012020740948FFF768FA0025002894
:1069800002D006E00220F8BD65613E600348FFF7D3
:106990005DFA2574F8BD0000E017002050C3000028
:1069A00011484168C9070BD0EFF3108172B60F4A46
:1069B000C2600F4AC26081F310884168C9070ED1D6
:1069C000416889070DD5EFF3108172B6094A02615B
:1069D000094A026181F310884068800701D50120CF
:1069E000704700207047000000200240EFCDAB89C7
:1069F00005040302BFAE9D8C1615141370470000EA
:106A000010B504494A69024202D04861FFF7F6FF17
:106A100010BD000000040140FCB500230124A2E0E9
:106A200027462A469F403A406FD04D68012D05D039
:106A3000022D03D0112D01D0122D16D18568032609
:106A4000AC465D00AE46AE406546B543AC46CE684A
:106A50007546AE4065462E43866046680D79BE4356
:106A6000ED06ED0F9D4035434560C6685F00032588
:106A7000BD40AE46AE4335468E68BE402E43C6602E
:106A80004E68022E01D0122E14D1DE08B600361840
:106A90000196366A5D07B446EE0E0F25B5400096A6
:106AA0006646AE43B4460D69009EB54066462E4329
:106AB000019D2E6206687546AE430D79AD07AD0F98
:106AC000BD40354305604D68ED004BD5294D6E6BDB
:106AD00026436E639E08284DB6007519AC46AD6816
:106AE0009E07360F0F27B740BD4305273F07B84223
:106AF00001D1002715E0214FB84201D1012710E054
:106B00001F4FB84202D102270BE02BE01D4FB842C5
:106B100001D1032705E01C4FB84201D1052700E051
:106B20000627B7402F436546AF60184D2E684F6863
:106B30009643FF0300D516432E606E684F68964358
:106B4000BF0300D516436E60AE684F689643FF02E0
:106B500000D51643AE60EE684F689643BF0200D57D
:106B60001643EE605B1C0A681546DA4000D057E712
:106B7000FCBD000000100240000001400004005075
:106B800000080050000C0050001C005000040140A0
:106B90000069084000D001207047426913460B404D
:106BA0001B0491430B4383617047002A01D081612C
:106BB000704781627047000001488068704700009C
:106BC0007801002002488168027889188160704746
:106BD0007801002010B508480024016840221143C4
:106BE0000160204600F00AF8002801D0012401E0ED
:106BF00000F042FA204610BD0020024070B5044665
:106C00000D4D7D202978C000FEF772FA01460B4831
:106C10000068FEF76DFA00F02BFF002809D1042C64
:106C200007D200222146401E00F04EFA00206C6080
:106C300070BD012070BD000078010020840100209B
:106C400070477047F8B502F01DFE604C0120E070FF
:106C5000208AFEF71AFD01467F20C005FEF718FBCB
:106C60005B4D06462968FEF7BAFA28600120A16A42
:106C7000C005814201DA084603E03046FEF704FB16
:106C8000A062FF21C9050025C84200D3A562607833
:106C900000280BD102214F48FFF77AFF02004E492E
:106CA0004E4817D00022FFF780FFE56202214948D5
:106CB000FFF76EFF4A4E002855D0E562B08AFEF716
:106CC000E4FC434F3968FEF7B7FD5FD24549012028
:106CD00008705DE00122D1034048FFF766FF208A7B
:106CE000FEF7D3FC01467F20C005FEF7D1FAE16A2A
:106CF000FEF775FA3C49E0628842D7DD3848012743
:106D0000F926403000900A213046FEF7F1F90029BB
:106D100003D131493148FFF701F902212D48FFF72E
:106D200037FF002801D0002701E0002F12D10221F7
:106D30002848FFF72DFF00280CD104F0A3FC009990
:106D40000120888005F0FAF9642003F013FD28493A
:106D50002648C8600A2003F00DFD3046761EF6B2C4
:106D60000028D0D1A2E7208AFEF78FFC01467F20C1
:106D7000C005FEF78DFAE16AFEF731FA1D49E062BF
:106D800088429BDB1A491948C86097E71548057087
:106D9000708F401EFEF76EFC3968FEF74DFD06D879
:106DA0002079002803D014490120087001E012481E
:106DB0000570708FFEF769FC3968FEF73DFD04D25F
:106DC0002079002801D004F021FCF8BD3C0100200E
:106DD00074010020000400500080000000000050FA
:106DE000E80D002076000020000040400400FA0575
:106DF00000ED00E00000A04086000020704770B564
:106E0000040010D0022025462035A873204601F04A
:106E100095FBA87B032805D0204600F0B9F8002098
:106E2000A873687370BD012070BD7047704710B5BE
:106E3000044600680168C943C90708D18168C9438D
:106E4000C90704D1012141602046FFF7FBFE2068FD
:106E50000168C943890708D48168C943890704D4F4
:106E6000022141602046FFF7EBFE20680168C9431C
:106E7000490708D48168C943490704D40421416003
:106E8000204600F0F7F820680168C943090708D4D4
:106E90008168C943090704D4082141602046FFF7EF
:106EA000ADFF20680168C943C90608D48168C94399
:106EB000C90604D4102141602046FFF7C2FE2068B5
:106EC0000168C943890608D48168C943890604D486
:106ED000202141602046FFF7A9FF20680168C943CF
:106EE000490608D48168C943490604D44021416059
:106EF0002046FFF79AFF10BDF8B5040005D02546DF
:106F00002035A87B002802D006E00120F8BD002033
:106F10006873204600F04EF80220A8732068C2680B
:106F200084466368012B01D10620824316486169BB
:106F3000814202D0072040038243002B01D1D82098
:106F400082431248A668024018463043676A266AA0
:106F50003E433043A66A30431043002B02D0012B3E
:106F600004D005E02369E2691A4300E0E2681043B7
:106F7000054A914202D0A269114308436146C860A4
:106F80000120A8730020F8BDFFFF0000F8F119FFF1
:106F900010B500680549884207D10548816B490052
:106FA000490881630D2000F073F810BD007C00409B
:106FB0000010024010B50068084988420CD108480A
:106FC000816BC20411438163002201210D2000F076
:106FD0007BF80D2000F06CF810BD0000007C004034
:106FE000001002400068C06970470000F8B5044610
:106FF0000220254620351746A8731D480268C304A1
:107000001A4302602068C2689B121A43C26020685B
:107010000269012632430261226810205060206814
:1070200081611021204601F0F9FA03281FD0216860
:1070300008204860206847610821204601F0EEFAE8
:10704000032814D0204601F079FAA87B03280ED03B
:1070500020688168314381602068016931430161A2
:1070600020680169042211430161AE730020F8BD5C
:1070700000040140704700000448416B01221143A5
:107080004163816B02041143816370470010024029
:10709000002809DBC106C90E0120884003490860A9
:1070A000BFF34F8FBFF36F8F7047000080E100E0A8
:1070B000002805DBC106C90E01208840014908608F
:1070C0007047000000E100E010B503F051F910BD79
:1070D00002494A6882434A607047000000700040DD
:1070E000024801688215114301607047007000403A
:1070F00002494A6802434A6070470000007000403D
:107100000548016802221143016004480169042214
:107110001143016130BF70470070004000ED00E096
:10712000F0B5154A1368154D54152D6A2340ED0727
:10713000ED0F002B04D0002D02D01668A643166078
:107140001668B608B600064316600D48076904269F
:107150003743076101290DD040BF20BF20BF01691F
:10716000B1430161002B04D0002D02D010682043F0
:107170001060F0BD30BFF2E7007000400000014039
:1071800000ED00E0F8B5044600780027534D800676
:1071900071D5524E403EB06BC00004D4B06BA9050F
:1071A0000843B06301274E480168C90511D401683E
:1071B000821511430160FFF7FFFC009005E0FFF727
:1071C000FBFC0099401A642837D845480068C00580
:1071D000F5D532680321090560680A4001409142F3
:1071E00008D08103890F032904D13168890301D5AF
:1071F0000120F8BD2A69032109040A4022D0084071
:1072000090421FD0207880061CD528692A698843BF
:107210000121C9040A432A612A698A432A61286133
:10722000C0050FD5FFF7C8FC009008E0FFF7C4FCCD
:107230000099411A2B48814201D90320F8BD2869E1
:107240008005F3D561688803800F032805D1326873
:107250000005824301400A433260286903226168C5
:107260001204114008432861002F04D0B16B0120A3
:1072700000078143B1632078C00705D0E868A168A2
:10728000800880000843E8602078800705D5E8681A
:107290000C218843E1680843E8602078400706D560
:1072A000E86803218902884321690843E86020785F
:1072B000000706D5E868032109038843616908438C
:1072C000E8602078000606D5E86803218904884331
:1072D000A1690843E8600020F8BD000040100240AA
:1072E0000070004088130000F8B50E46050038D045
:1072F0005E480068C007C00FB04214D25B4C2068E3
:107300004008400030432060FFF756FC074605E088
:10731000FFF752FCC11B564881427AD82068C0074B
:10732000C00FB042F4D12878524C800705D5E068F0
:10733000F0218843A9680843E0602878C00752D04C
:107340006868022806D0032807D0216801280AD0DF
:10735000890504E02168890301E021688901002989
:1073600003DB0120F8BD4907F9E7E16889088900D6
:107370000143E160FFF720FC0746686802280AD055
:10738000032814D001281ED029E0FFF715FCC11BEB
:10739000374881423DD8E0680007800F0228F4D1C9
:1073A00021E0FFF709FCC11B3148814231D8E06878
:1073B0000007800F0328F4D115E0FFF7FDFBC11B88
:1073C0002B48814225D8E0680007800F0128F4D1BE
:1073D00009E0FFF7F1FBC11B2548814219D8E0689D
:1073E0000007800FF5D121480168C907C90FB142D4
:1073F00017D901684908490031430160FFF7DCFBF8
:10740000074608E005E0FFF7D7FBC11B184881429B
:1074100001D90320F8BD15480068C007C00FB0426D
:10742000F1D12878400706D5E06807210902884392
:10743000E9680843E0602878000707D5E06807217D
:10744000C90288432969C9000843E06000F03AF89E
:10745000E168094A0906090F515CC84007490860FC
:1074600007480068FFF7CAFBF8BD00000020024093
:10747000881300000010024016C300088401002099
:107480007C010020044805490068C968044A490590
:10749000490F515CC8407047840100200010024031
:1074A0002FC30008044805490068C968044A8904D4
:1074B000490F515CC8407047840100200010024011
:1074C0002FC3000870B51A4AD3681A490C20184017
:1074D0008D0004280CD04E00082810D00C2810D0A5
:1074E00050680004410F0120C003491C884070BD52
:1074F0001068C00601D5084670BD284670BD3046EC
:1075000070BD98020C4C000F205C1B029C0FD368CE
:10751000641CDB0301D5314603E01268D20600D4B7
:10752000294602F0EAFE22460023FDF7F7FD70BD72
:107530000010024000093D0026C30008FEB505000A
:107540007ED0FE4CE7680C20E6680740012000046E
:1075500006402878C00747D0082F05D00C2F0AD145
:1075600001200004864206D1206880033CD568686B
:107570000028E5D038E0012069680004814203D189
:1075800021680143216011E0052301221B049204BC
:107590009942216802D111432160F1E781432160C2
:1075A00021680140009120689043206068680028AD
:1075B0000DD0FFF701FB009005E0FFF7FDFA009901
:1075C000401A64287BD820688003F6D50CE0FFF7CA
:1075D000F3FA009005E0FFF7EFFA0099401A6428EB
:1075E000F0D820688003F6D42878800756D5092380
:1075F000E868042F0DD00C2F01D1002E09D00028EF
:107600003CD02168994301432160FFF7D5FA064633
:1076100028E02168490701D5002891D061681F2220
:10762000120291432A691202114361602168994351
:1076300001432160FFF746FFE16809060A0F00E0F9
:107640008BE1BF49895CC840BE490860BE480068FC
:10765000FFF7D4FA002873D120E0FFF7ADFA801BC2
:107660000228AFD820684007F7D560681F210902BB
:10767000884329690902084360600FE020684008D8
:1076800040002060FFF798FA064604E0FFF794FAFE
:10769000801B022896D820684007F7D42878C006B7
:1076A00060D5002F0CD0A86900284AD02068FF219F
:1076B000013108432060FFF77FFA06462EE0C1E063
:1076C0002068800502D5A8690028A6D06068072137
:1076D00049038843296A084360606068297F000283
:1076E000000A090608436060286A410B0120C003B4
:1076F000491C8840E16809060A0F9149895CC84025
:107700009049086090480068FFF778FA002817D180
:1077100028E0FFF751FA801B0228A2D820688005D4
:10772000F7D56068072149038843296A08436060E8
:107730006068297F0002000A09060843606011E0C2
:10774000E2E02168FF20013081432160FFF734FA35
:10775000064604E0FFF730FA801B022872D8206842
:107760008005F7D42878794E000724D56869002869
:10777000306910D0012108433061FFF71DFA0090F5
:1077800005E0FFF719FA0099401A02285AD8306923
:107790008007F6D50FE0400840003061FFF70CFA93
:1077A000009005E0FFF708FA0099401A022849D82E
:1077B00030698007F6D42878400766D5002002900B
:1077C000A06BC00006D4A06B012109070843A06389
:1077D000012002905E480168C90511D40168821534
:1077E00011430160FFF7E8F9009005E0FFF7E4F9C5
:1077F0000099401A642825D855480068C005F5D579
:10780000FF20AA680130824203D13169014331610E
:1078100011E001218902002A07D005231B029A42A8
:1078200003D132690A433261EFE732698243326140
:10783000306988433061A868002810D0FFF7BCF990
:10784000009008E05FE0FFF7B7F901460098091AD9
:107850004048814257D830698005F4D50DE0FFF7E4
:10786000ABF9009006E0FFF7A7F90099411A3948F3
:10787000814248D830698005F5D40298002804D0A8
:10788000A06B012109078843A063686A002866D0BD
:107890000C2F3ED0012636060228206805D0B043C2
:1078A0002060FFF789F905462FE0B0432060FFF71D
:1078B00083F9074604E0FFF77FF9C01B022822D8AE
:1078C00020688001F7D4E96AA86AE2680843296B56
:1078D000FD231B049A4311430843E06020683043B2
:1078E0002060FFF769F9054604E0FFF765F9401BE2
:1078F000022808D820688001F7D530E0FFF75CF94E
:10790000401B022801D90320FEBD20688001F5D468
:1079100025E00128F8D0E06801210904AA6A0140A5
:1079200091421AD10F218904EA6A0140914214D18F
:10793000032189050840296B88420DE000100240B0
:1079400016C30008840100207C0100204010024082
:10795000007000408813000001D00120FEBD00200F
:10796000FEBDF8B504000ED0FF27606A053700257C
:1079700000280AD02561656126464036A562707CE4
:10798000002807D00AE00120F8BD6068B842F3D0B3
:10799000E561F1E73574204600F03EF8022171748C
:1079A0002068026840239A4302602123A26860682D
:1079B0009B021A4038401043E3688A021340184380
:1079C00023690B40217D1843C907C90F0843A169EA
:1079D000931019400843E169382319400843216A8C
:1079E000802319400843A16A930019400843216885
:1079F0000860A0690421000C0840616A1023194046
:107A00000843216848602068C1699143C161656588
:107A1000012070740020F8BD10B586B00446142112
:107A20006846FDF7C4FB10492068884219D10F4809
:107A3000416B821411434163C16A01221143C16247
:107A4000C06A002110400590E020009002200190C3
:107A50000320039002910491052069460007FEF778
:107A6000DBFF06B010BD00000030014000100240F6
:107A7000094910B5401E884201D9012010BD074CAC
:107A800060610321081F02F073FC0020A061072041
:107A90002061002010BD0000FFFFFF0000E000E0BB
:107AA00070B505462C4602202034002908D0042950
:107AB0000BD008290ED0627F012A10D0012070BDA2
:107AC000A27E012AFAD1A0760AE0E27E012AF5D14F
:107AD000E07605E0227F012AF0D1207700E0607790
:107AE0000122286801F044FF012228689207012141
:107AF000904205D0074A904202D0074A904204D1F2
:107B000082685207520F062A02D002680A430260B6
:107B1000002070BD000801400014014070B504460B
:107B20000D460068002201F023FF2068016A0C4A1C
:107B3000114203D101684908490001600120203445
:107B4000002D06D0042D06D0082D06D06077002029
:107B500070BDA076FBE7E076F9E72077F7E7000055
:107B6000111100007047704770470000F8B50268B7
:107B70000446D06911689668814B05461D40202354
:107B8000002D6CD0F7077F4DFF0FBC460D402F43F3
:107B900079D02546C7078035002F06D0CF0504D5FC
:107BA000012717622A683A432A60820708D5F2073C
:107BB00006D0276802223A622A6804273A432A60DC
:107BC000420708D5F20706D02668042232622A68E6
:107BD000022632432A6002070AD50A461A40664640
:107BE000324305D02668082232622E6816432E6082
:107BF000020508D54A0106D501222668D202326262
:107C00002A681A432A602A68002A30D0800606D5DE
:107C1000880604D5616E002901D02046884728686F
:107C200021688968490602D42821084225D02046C7
:107C300002F0AFF820688168490619D582684021B2
:107C40008A438260206F002812D04F498163206FE1
:107C5000FEF748FD00280AD0206F816B06E08506FC
:107C600011D58D060FD5616E77E020468847F8BDA7
:107C70002046FFF779FFF8BD05E02046FFF774FFC7
:107C800000202860F7E7256E012D56D1C50654D592
:107C9000CD0652D510261662206881682546490611
:107CA000403500292ADA226F116849680904090C55
:107CB000E1D02F8B8F42DED969831168096889066C
:107CC00017D4016832019143016020688168490836
:107CD0004900816020688168402291438160E367A8
:107CE0000020206620680168B1430160206FFEF724
:107CF000D7FC288B698B401A81B21AE0298B6A8BDA
:107D0000891A6A8B89B2002AB5D00029B3D00268DB
:107D1000FF252135AA43026020688268520852007C
:107D20008260E36700202066606620680268B243D4
:107D300002602046FFF716FF9DE7C50208D57502D1
:107D400006D50120000510622046FFF70CFF92E7E0
:107D5000050605D50D0603D5A16E002985D18AE754
:107D6000400688D5480686D5116820464024A143A0
:107D7000116083670021816600F043F97BE7000012
:107D80000F08000020010004B99C000810B5040091
:107D900003D0A06F002802D007E0012010BD002111
:107DA00074200155204600F027F82420A0672068A1
:107DB0000168490849000160204602F03DF80128A9
:107DC000ECD0606A002802D0204601F05FFE2068F7
:107DD00041680922D20291434160206881682A22C9
:107DE00091438160206801680122114301602046AF
:107DF00001F0B2FE10BD0000F0B587B006461421B8
:107E00006846FDF7D4F92C493068884251D12B4897
:107E1000416B0122920311434163C16A0122114364
:107E2000C162C06A00251040059003204002009006
:107E30000220032701A9A1C104200490052069465E
:107E40000007FEF7E9FD1F4C1D48A560E56081C4F1
:107E50008027E560A7602020256160610002A061A5
:107E60001848083CFEF7B8FC002801D0FDF76AFF6F
:107E70003467A662144C124821461438206003204F
:107E8000606010200831A1C16561A561E5612046EF
:107E90002562FEF7A1FC002801D0FDF753FFF46630
:107EA000002201211B20A662FFF70EF91B20FFF71D
:107EB000FFF807B0F0BD000000380140001002409C
:107EC00030000240501700209817002070B5C36F93
:107ED000202B27D100290BD0002A09D00124836848
:107EE0002403A34206D10369002B03D1CB0701D0A1
:107EF000012070BD034660331C7D012C12D001248B
:107F00001C7500230366084C0368A34207D05C6815
:107F1000240204D51C680125AD062C431C6002F028
:107F20008BF870BD022070BD00480040704770475C
:107F3000FFB50446806F83B017460D4620285ED1FA
:107F4000002D0AD0002F08D0A168C001814207D1BE
:107F50002069002804D1E80702D0012007B0F0BD55
:107F6000204660300090007D012848D00098012113
:107F700001750020802108512120A067FEF71CFE1A
:107F8000264640360190378277820120A16800039F
:107F9000814202D12069002805D02F460025009992
:107FA0000020087511E00027F9E700228021204613
:107FB00002F088F8002815D1002F15D021683878F4
:107FC00088627F1C708A401E7082708A019B002824
:107FD00006980090E9D100224021204602F072F874
:107FE000002808D00320B9E728882168C005C00D03
:107FF0008862AD1CE6E72020A0670020AEE70220E3
:10800000ACE77047034D044C04A002F055F9E5605D
:10801000FAE700000400FA0500ED00E04861726430
:108020004661756C745F48616E646C65722E0D0AF2
:108030000000000070B586B014216846FDF7B7F85F
:1080400001240B480C4EC4800A48A50244832246F2
:1080500029463046FEF7A9FD0021029103910095C3
:10806000019469463046FEF7D7FC06B070BD0000AB
:10807000280E00203C0100200004005010B505240B
:108080002407002204212046FEF78FFD002208214C
:108090002046FEF78AFD0A2002F073FB012204212C
:1080A0002046FEF782FD0A2002F06BFB002204212D
:1080B0002046FEF77AFD10BD10B5052424070022E6
:1080C00004212046FEF771FD012208212046FEF71B
:1080D0006CFD0A2002F055FB012204212046FEF728
:1080E00064FD0A2002F04DFB002204212046FEF729
:1080F0005CFD10BDF8B50024052607462546360769
:10810000002204213046FEF750FD0A2002F039FB20
:10811000012204213046FEF748FD6006040E0821C6
:108120003046FEF735FD002801D0641CE4B205207E
:1081300002F027FB6D1CEDB2082DE1D3002F03D018
:10814000FFF79CFF2046F8BDFFF7B6FFFAE770B5D2
:10815000052605463607002204213046FEF725FD98
:108160000024E80901D0012200E000220821304665
:10817000FEF71BFD6806050E0A2002F002FB012235
:1081800004213046FEF711FD0A2002F0FAFA00221F
:1081900004213046FEF709FD0A2002F0F2FA641CC1
:1081A000E4B2082CDDD370BD10B5052424070122EC
:1081B00008212046FEF7F9FC012204212046FEF7A3
:1081C000F4FC002208212046FEF7EFFC0A2002F012
:1081D000D8FA002204212046FEF7E7FC10BD10B5B6
:1081E00005242407002204212046FEF7DEFC00229D
:1081F00008212046FEF7D9FC0A2002F0C2FA01222B
:1082000004212046FEF7D1FC012208212046FEF77A
:10821000CCFC0A2002F0B5FA10BD70B505252D077B
:108220000024012208212846FEF7BFFC062002F0A8
:10823000A8FA012204212846FEF7B7FC062002F026
:10824000A0FA07E0641CE4B2FA2C03D9FFF7C7FFD9
:10825000012070BD08212846FEF79AFC0028F1D1C4
:10826000002204212846FEF7A0FC002070BD00007B
:10827000F8B501F0A3FC01F0D3FC5B480068C069CD
:10828000FDF750FE594C0246A08259480121808FCB
:108290008902584E0025002843D0A36A4F03564850
:1082A000BB4202DB0223037000E005700078002867
:1082B00005D001280ED0022810D003281DD1608BD4
:1082C00001282ED0022818D1474808214038FFF74E
:1082D00025FC12E0FF20F5308242F0D2608B0128AD
:1082E0001DD0022804D008E03046FEF75EFC04E012
:1082F0003D4808214038FFF7D3FBFDF71DFF2070F4
:108300000121C9023046FEF743FC0127FF03002884
:108310002DD03A480560A079002804D007E001225A
:10832000E2E70022E0E70120A07101F02DFF8021AB
:108330003046FEF72DFC002806D0002208213046EA
:10834000FEF733FC012205E0012208213046FEF74A
:108350002CFC0022052039460007FEF726FC244CA1
:10836000274E4034A08C274F012803D01CE0A57174
:108370000022EAE724486946088072B68021234833
:10838000FDF7F8FC002804D0022269461F48FDF7DB
:1083900095FD62B61EA001F08FFFA58403F0CEFE0E
:1083A000642002F0E7F9FE60608C012808D11048D3
:1083B0006584058003F0C2FE642002F0DBF9FE60F4
:1083C000208C012806D1258403F0B8FE642002F039
:1083D000D1F9FE600648124A0188914202D1C08854
:1083E000002800D1FE60F8BDCC1600203C01002022
:1083F000E80D0020000400508400002074010020DB
:108400000400FA0500ED00E0AAAA0000384A0008BE
:10841000BDF8C8EBC9FDBCB6C4A3CABD0D0A0000B7
:10842000AA55000038B55721202000F07AF8032122
:10843000212000F076F84021222000F072F8082177
:10844000232000F06EF8AA21302000F06AF81048CE
:10845000018F142901D8002901D1012101870C4C79
:1084600040346188142901D8002901D1022161809A
:10847000008FC1B2322000F054F8A178332000F010
:1084800050F8684600F006F80A2002F07AF938BD84
:10849000E80D002010B501460F2000F021F800285B
:1084A00000D0012010BD10B50446FFF77DFE32203C
:1084B000FFF74DFEFFF7B1FEE0B2FFF748FEFFF712
:1084C000ACFEFFF771FE3320FFF741FEFFF7A5FE7C
:1084D0000020FFF70FFE0446FFF781FE204610BD87
:1084E00010B50C46FFF7DFFF2070012010BD70B5FE
:1084F0000D460446FFF758FE3220FFF728FEFFF72F
:108500008CFEE0B2FFF723FEFFF787FE2846FFF759
:108510001EFEFFF782FEFFF762FE0A2002F031F92D
:1085200070BD10B5FFF7E3FF012010BD10B5024884
:10853000FEF77DFC10BD000004160020FEB50446C9
:10854000002772B6334A01688B1804D13248C768D5
:1085500003208004074088680190C868009048693B
:108560008E69002B08D12C4940398B6ACD042B43EE
:108570008B628B6AAB438B62014631433CD0254909
:108580002368CB4205D12449CA6803239B049A433C
:10859000CA6025462035002810D021680A690123C9
:1085A0001A430A61216848610821204600F036F824
:1085B000032800D1A873216808204860002E10D03D
:1085C0002068016901221143016120688661102140
:1085D000204600F023F8032800D1A873216810205A
:1085E00048600C482168C14206D10B48C16803228B
:1085F000920491433943C1602068016949084900E8
:10860000016121680198886021680098C86062B69D
:10861000FEBD00000084FFBF4010024070B506465A
:108620000B480D46002409490068FCF761FD7D21D7
:10863000C90048433168401E00D103240B682A4614
:108640009A4301D00028F6D1204670BD204E00008C
:10865000840100201CB5002116480091144A0191A4
:108660000260C163120542608160072282630122B9
:1086700002610246C16020321170FF235170C23383
:10868000436281621173016381610422416342612B
:10869000C161FDF76BFE08480090801301906946A8
:1086A0000448FDF713FE00210248FDF7B9FD1CBD8B
:1086B00000240140A81500200200000408B5084865
:1086C000016B012211430163006B012110400090F6
:1086D00000220A20FEF7F8FC0A20FEF7E9FC08BD9C
:1086E00000100240F0B587B014216846FCF75FFD2A
:1086F0004B48C26A04210A43C262C26A0A40059218
:10870000C16A80273943C162C16A39400591C16A93
:1087100001252943C162C16A29400591C16A022627
:108720003143C162C06A2A463040059005201C21B1
:108730000007FEF73AFA01223A493B48FEF735FABC
:1087400000223A493848FEF730FA912105200022EC
:1087500009020007FEF729FA354801900024052098
:108760006946009502940007FEF756F90C20009028
:108770001120019003200390052002946946000710
:10878000FEF74AF9102000900520694603960195EE
:1087900002940007FEF740F9112001900294694607
:1087A000009503942048FEF737F922480190694666
:1087B000009602951C48FEF72FF9E8026A4651C25E
:1087C00069461948FEF728F91B480090029469464B
:1087D000019503941448FEF71FF920206A4631C220
:1087E00069461148FEF718F9912000020090052013
:1087F00002946946019503940007FEF70DF9694656
:108800000948009702950194FEF706F9002201211C
:108810000520FEF759FC0520FEF74AFC07B0F0BD25
:108820000010024001020000000400500830000067
:1088300000001110000021100832000010B50F4C8C
:108840000D482060FF20053060600020A060E060DF
:1088500020616061E0610121206249026062A161E2
:10886000A0620720E0622046FFF77BF820680168DD
:1088700040221143016010BD003001403416002039
:1088800000B585B014216846FCF791FC0E480D49EF
:108890000160E1214902416000218160C160016104
:1088A00081610C22C161426101623021416201217A
:1088B000090381634900C163FFF768FA01F05EFCB8
:1088C00005B000BD00380140CC1600207047000004
:1088D000F0B589B00A2002F09FFC7D20400102F033
:1088E000B5FCFD4C0025A570FC482066607C0C287A
:1088F00001D30B20607460790A2801D90A206071C5
:10890000E5702021F648FEF743F9002862D00020E8
:10891000F449A076F44E09783171F44AA1791278BD
:1089200049001143A27DC000920011430143F1713F
:10893000E06BF070010A3172401CE0636079B07442
:1089400042003046EA491330FCF718FC6079E849E8
:1089500082004000801960311330121DFCF70EFCBC
:1089600060790621420048438019E2491730921C81
:10897000FCF704FC3020205E002803D0DE49098A81
:10898000081820866079D449C000203182190B7CF8
:1089900053764B7C937606227272D84A1D30127839
:1089A000B272E28C3273D04A0B7A133A1375497A59
:1089B00051750022CC4902F019FD60790021C000F8
:1089C0001D3002F025FDCE48FEF70CFB0127608527
:1089D000BF030BE001209BE7C948FEF703FB80B211
:1089E0006085218FFF392D39884206DB218F80B2C7
:1089F0008842F1D3C9198842EED8022002F05CFC0B
:108A0000B9480126C571A574A5732674E573BC48E1
:108A1000FEF7E8FAA0850746E5706079FCF750FE9E
:108A2000B84AB94BFCF730FD01F040FE0022B74BCD
:108A3000FCF778FCFCF78AFE0006C00CC01980B277
:108A4000F103E085884201D3401AE085B048E06434
:108A50002079401C2071AA48FEF7C4FA6085A4481A
:108A60009D4F643840370690B2E1A548FEF7BAFA48
:108A700060850BE0A248FEF7B5FA80B26085E18D13
:108A8000884203D3A34A8918884207D300210F20C4
:108A900002F042FBA04920640842EBD0206C411C4C
:108AA0001FD040047ED58122D20100210F2002F088
:108AB00072FC0021102002F02FFB41068C48490E69
:108AC00000227C38E16502F05DFB002002F0BEFB75
:108AD000002002F070FB86487C38417A0729C3D118
:108AE00001E001F067FC02228C49401DFCF76AFBA3
:108AF0000028B9D102F0DDFCE167A06702F0C6FCF6
:108B0000754B803303C3E0787949401CE0708339AA
:108B10000B7A68460370497A417000880390218D72
:108B200088427DD170497E488C31C98E01806E4962
:108B300069488C31098F81847148FEF753FA60854A
:108B400002F0FCF96448FF2280300168406852045A
:108B50000023891858410206080A104341084900B9
:108B600000900A0E08025C498031CA6088605E4845
:108B7000E36F0A30A26F02F071FC607981005A48FD
:108B800008185549163080310CC902F067FC52486C
:108B90008030C36882685448123002F05FFC0821BC
:108BA000514800E007E14172B430C07C00096075B3
:108BB00014D04F48022259497738FCF703FB0028AC
:108BC0000CD14948A674C671E06D49491638C2B245
:108BD0006639C81DE274FB30FCF7D0FA60790022D8
:108BE000800041491C3002F001FC607900218000C6
:108BF0001C3002F00DFC009802F007FB012002F08F
:108C00005BFB207302213648FDF7C2FF00281DD010
:108C100000213648017034488C30418E049100E0C8
:108C200082E03981808E788184463149A06C603140
:108C3000E0640860DC392065C97C0907090F032955
:108C400000D02175E16D1C2902D015E00121E0E77B
:108C50002549214A8C31C98F5186069B254A1B889C
:108C60001380884207DD002805DD002903D0207E1F
:108C7000401C207600E025762571A6730498B88103
:108C80006046F881E673A08C2649FF30C33080B27D
:108C9000A08488420CD949424018A08420487D22F3
:108CA0000188D200491C89B20180914200D305801D
:108CB0001B487D210088C9004843A18C401860658D
:108CC00000F07CFD207B002805D100210F2002F060
:108CD00023FA0006F9D584E0700000203F420F001F
:108CE000000400503C0100205C12002070010020B4
:108CF0008C130020C8140020280E00204C010020F6
:108D000004160020B81E85EB51B8CE3F0000084085
:108D1000A0860100983A000000D0272460010020BE
:108D20006C010020E7030000FDF7E4F8684A032126
:108D3000115468494A8E3A81898E7981E26D1C2AE4
:108D400006D1634B4200AC33D318069A12885A807E
:108D500080005F4A5F4B603A02905D4982189B8FAA
:108D6000138030394118A26C4A605A498C39401836
:108D7000594916300CC902F071FB216EA06C884273
:108D800008DA534A0299603A5158012902D1206603
:108D9000039905914E49029A60398A58824217DD3B
:108DA000012A15DD2146002812DD039808850220DE
:108DB000087065730CE0494A00210F2002F0EBFABD
:108DC0006079E178401C814202D0002002F0F3F982
:108DD000608DE18D884200D247E6414A8918884279
:108DE000FAD8A07B012801D00220A07302F0A6F8D7
:108DF0003A4A00210F2002F0CEFA2079002817D03D
:108E0000384909888A008B18834200D225700020D7
:108E100000F0E2F8A07C002839D02D490C310B7805
:108E2000A372487860728A782272022B17D02EE0E3
:108E3000E16C226E323920468A420EDAC179294A23
:108E4000491CC9B2C171128852008A42E2D2059906
:108E50000185022101706573DCE7E571DAE710280E
:108E60000CD0C82813D2204BC91C1818FCF786F95F
:108E700003F064F9642001F07DFC32E61B4D2868A4
:108E80004000000E03D1C878FCF7FFFB28600020EB
:108E90002378627B65790FE00D4E4100903E775A52
:108EA0001836765AB74205D00A4F0223002201260F
:108EB0008C377E52401CC0B2A842EDD3237062733F
:108EC000064A002180320F2002F065FA09B0F0BD99
:108ED0001C140020E8120020F000002000D02724FD
:108EE000983A00004C010020E80D002064010020A9
:108EF000F8B52E4C0546E06E2D4A281A411E206713
:108F0000914215D21C21615E081AFCF7C5FB294A63
:108F1000294BFCF7B9FA064634200F46205EFCF7D1
:108F2000BBFB32463B46FCF7FDF9FCF7EBFBA086AA
:108F3000002060761D481E23C35EC28C1F48008837
:108F400084461F4806881DE06046484380181D4F30
:108F500080B23880302778436427643078431A4FD2
:108F60006066C01985420BD2C8B218493422088005
:108F7000606EA25E411BC9188918A166E066F8BD43
:108F8000491C6176617EB142DED3302042431048F5
:108F90006421101848430F494118E1666066342186
:108FA000401B615EC0184018A066F8BD700000202C
:108FB000CF0700009A9999999999B93F5A010020D1
:108FC0004C0100206E01002078ECFFFF58010020CA
:108FD00074270000C0BDF0FFFEB5294D2988491C4B
:108FE0008FB228492F800E88FCF756FB264A274B64
:108FF000FCF74AFA0191009025483146FCF778F8D1
:10900000244C618F4218B74206D3002028802248A2
:10901000019E1018009D02E01046019E009DFCF785
:109020004FFB33462A46FCF77DF9FCF78FFBE086C1
:10903000012580B2ED03A84201D3401BE086208CBD
:10904000FCF73EFB154A164BFCF786FA0646E08E07
:109050000F460090FCF734FB32463B46FCF762F9C2
:10906000FCF774FB80B22087A84201D3401B208705
:109070000C4900980968486100986087FEBD0000AF
:10908000580100204C0100201904560E2D6240406A
:10909000E17A0000700000201F050000F853E3A5EE
:1090A0009B843E400416002070470000F0B589B054
:1090B000002004900A2002F0AFF87D20400102F069
:1090C000C5F8B34800228270C16BB34C491CC16320
:1090D000B049038E098A2546C91801862146C27502
:1090E00013310791473103916D393135AB4F203042
:1090F00005910290A64E0F21A94871710078207148
:10910000A84AB079127840001043B27D9200104313
:10911000E071B08FE070000A2072A17431461E2207
:109120009C310798FCF72AF8402228469E49FCF714
:1091300025F8029903980A7CC274497C01750920BC
:1091400060729A480078A072F08C2073F07D410024
:1091500030469C30091805980A780275497841759F
:10916000762000228C4902F041F9707906214843AB
:1091700000211C3002F04CF9022002F09DF8002181
:109180000F2001F0C9FF38423064F8D0306C411C28
:1091900018D040047ED58122D20100210F2002F098
:1091A000FAF80021102001F0B7FF41067A48490E75
:1091B0000022B43001F0E6FF7748B430417A02294A
:1091C00002D0BDE001F0F6F802227949401DFBF71C
:1091D000F9FF0028F5D16E480222C07D41006C489D
:1091E0009C3009186C48B530FBF7ECFF0028E8D13B
:1091F00002F05FF9664AD167906702F047F9644A66
:10920000803203C2049800282CD1012004906248C7
:10921000684E8C30C08E604930805D488C31098F3B
:1092200081846548FDF7DEFE5949644A4885888C8B
:10923000FF30C33080B2888490420CD952428018EB
:10924000888430885D4A401C80B20B323080904266
:1092500001D30020308030887D22D20050438A8C98
:10926000801848654C4869468C30428E0A80808E52
:10927000488049490422B531C81FFF38FBF77EFFFB
:109280004348494AC07D00998000115040498031CF
:1092900003C900E075E0FF235B040022C0185141C0
:1092A0000906060A0E43304601F0AFFF7108490077
:1092B0000A0E0802364900268031CA6088603448A8
:1092C000C36F826F3448483802F0C8F830488030A5
:1092D0000CC83148443802F0C1F82D488030C368CA
:1092E00082682D48403802F0B9F82B4900225239E3
:1092F0003C2002F07BF800213C2002F089F801209C
:1093000001F0DAFF2249087308468078401C887013
:1093100001210520C9030007FCF700FE1C48007B63
:10932000002805D100210F2001F0F6FE0006F9D536
:10933000802200210F2002F02EF81548467002E02E
:109340001349012048701248C17D491CC9B2C1753A
:109350000F2900D2CEE60498002810D10C4A1849F3
:10936000D08C002802D00B88984201D90888D0847C
:10937000144980B20988401E48431349088009B047
:10938000F0BD124A00210F2002F005F8D8E70000D6
:1093900070000020280E00205C12002000D027243E
:1093A0003C01002070010020781400204C010020B6
:1093B000600100206C01002004160020E70300007B
:1093C000480100204601002044010020009027248D
:1093D000F8B531492F48086002F054F92F4800F0E1
:1093E000ADF92F4CE0822D48801C00F0A7F92083B6
:1093F0002A48001D00F0A2F960832A482C214180F0
:10940000014640310979284F0906090E617006D1DD
:10941000C7800121C1870A21418700218187234A12
:10942000C18E1170C18F2171818F6171817AA1709C
:109430008588052165626181C6883046FBF758FE44
:10944000A08101462846FBF753FE8800081885B224
:10945000154825816843FCF733F9154A154BFCF78D
:109460007BF8FCF773F9E081658231463846FBF7FB
:109470003FFE20820146C820FBF73AFEE083012030
:10948000A083FCF74FFDA082E2890B490B48FDF752
:10949000ADFDF8BDA9A1000868000020004F00083C
:1094A0003C010020E80D0020E80300001800002027
:1094B000F853E3A59B843E40FF7F00000416002084
:1094C000F8B57B4C00267B4D2671012028807A4917
:1094D000C8200880E07A794F401CE072202138468D
:1094E000FDF756FB00285CD00020A076E07AC0078C
:1094F00006D0E18C481EE084022901D2C820E08415
:109500000120C043FFF768FD0A2001F085FE7D20A1
:10951000400101F09BFE02213846FDF739FB00288F
:1095200041D00020664980000978674F4900084310
:10953000644909780843B872102078726348C1887A
:109540007D20C000FBF7D4FD787361485F4A007846
:10955000B87338460B3091780170D17841705B490F
:10956000421C20310B7ED370497E11715749D01CAB
:1095700022310B7E5371497E9171544940310A7CEE
:109580000271497C417100223946172001F02EFFFB
:109590000021172001F03CFF022001F08DFE4D4F0D
:1095A00005E00120A1E70120BCE7FEF761FE0021F4
:1095B0000F2001F0B1FD38422064F6D0206C411C30
:1095C00073D040046FD58122D20100210F2001F019
:1095D000E2FE0021102001F09FFD41063A48490EAD
:1095E0000022B430E16501F0CDFD374FB437787A11
:1095F000112858D102223849781DFBF7E3FD0028D5
:1096000051D1F81F027A69460A70407A4870B97AD7
:109610002980C820FBF76CFD2749304D0880387B36
:10962000E08438462838C08E2880394620482839BA
:10963000098F81842A48FDF7D5FC6085A08C2949D3
:10964000FF30C33080B2A08488420BD94942401811
:10965000A08428882349401C80B20B31288088428E
:1096600000D32E8028887D21C9004843A18C401852
:10967000606500F0A3F86846008820851249B87C30
:10968000C7316071420008460D466930FBF776FD30
:109690006079294642001448FBF770FDE08CFF28F2
:1096A00001D003202070F8BDFFE700F083FE00002A
:1096B000700000204C0100205A01002000040050DE
:1096C00040010020410100205C120020E80D002034
:1096D0001800002000D02724600100206C01002029
:1096E00004160020E7030000A413002070B586B024
:1096F00014216846FBF75BFD01250F4EED030022A8
:1097000029463046FDF751FA0120002401900294C9
:109710006946009503943046FDF77EF903200190D9
:1097200002946946009503943046FDF775F90220CE
:1097300001F020F806B070BD0004005000887047AA
:1097400070470000F8B5044600206A461080194DA5
:1097500055222A70AA226A700322AA70661DEE7032
:109760002A716971144A49008918AC712246E81DB2
:10977000FBF704FD002007E029186A468978128863
:1097800089186A461180401CB042F5DB611DA81C97
:10979000FCF728FA01466846018029190078C8714B
:1097A00068464078087221460931024800F012FBF1
:1097B000F8BD000042150020E80D0020FEB5FFF7BF
:1097C00097FB2548FDF70EFC244C86B26685607930
:1097D0000A21081AC000FBF75FFF07460191A06E3F
:1097E000FBF76EFF1E4A1F4BFBF7B6FE00900D46BF
:1097F0003046FBF765FF2B46009AFBF793FD3A4690
:10980000019BFBF78FFDFBF7A1FF85B2E586208C5E
:10981000FBF756FF124A134BFBF79EFE06460F4618
:109820002846FBF74DFF32463B46FBF77BFDFBF737
:109830008DFF81B20120C0032187814201D3091A23
:109840002187854201D3281AE0860349E08E096802
:1098500048616087FEBD00000416002070000020F3
:10986000F853E3A59B843E40034A1168382389B22C
:1098700099430143116070470030014010B5FDF776
:10988000A1F910BD10B59AB034216846FBF78FFCE2
:1098900014210DA8FBF78BFC1C2112A8FBF787FCF9
:1098A0001B4801680324E402A143C2148918016023
:1098B000FDF716FC17480169A143016106200090DD
:1098C000FF2001300290012003901020049002201C
:1098D000099040040B90000100240C900A94684603
:1098E000FDF72CFE0F200D9003200E900F94109486
:1098F000012111940DA8FDF7F7FC8120129003209F
:1099000080041890149412A8FDF73CFC1AB010BD06
:109910000070004040100240104801688215114359
:109920000160C1680E4A1140C16001680D4A1140D2
:109930000160816849084900816001680122920440
:1099400091430160C168FD2212049143C16000216E
:109950000161064904488860704700000010024019
:109960000C40FF88F6FFF6FE0050000800ED00E016
:1099700010B5CB06DB0E0121046A99408C430462CA
:10998000016A9A401143016210BD0000F8B510242D
:1099900005252D07AC62AF20800000F0F2FEAC611F
:1099A00001F0CEFB2F4C304F304E60670EE001F0DF
:1099B000C7FB6067FEF75CFC606C411C61641428A7
:1099C00004D92BA000F078FC2D48C760606FB0422E
:1099D000EDD10026666420780127FF03030000F024
:1099E000A4FC05040C192D3032000122394628460A
:1099F000FDF7DBF8FFF764FD06E001223946284653
:109A0000FDF7D3F8FFF752FB002239462846FDF751
:109A1000CCF818E0607B0122401C60733946284670
:109A2000FDF7C3F8FCF79AFA002239462846FDF7FD
:109A3000BCF8607B052806D9267004E0FEF748FFD5
:109A400001E0FFF733FB02210E48FDF7A1F80028E3
:109A500005D000200C49087001F058FAF8BD01202B
:109A6000F8E70000700000200400FA053001CADEAB
:109A70004457204944204552524F522E0D0A0000AF
:109A800000ED00E0000400507001002010B5818C52
:109A9000C90707D001684A6801235B049A43836AB7
:109AA0001A434A60818C890707D501684A680123F7
:109AB0001B049A43C36A1A434A60818C490707D53D
:109AC00001684A6801239B049A43036B1A434A6066
:109AD000818C090707D501684A680123DB039A4393
:109AE000436B1A434A60818CC90607D502689168A6
:109AF00001231B039943836B19439160818C890671
:109B000007D501688A6801235B039A43C36B1A4334
:109B10008A60818C490612D503685A6801210905BB
:109B2000046C8A4322435A60026C8A4207D102685D
:109B3000516803235B059943436C19435160818C41
:109B4000090607D501684A680123DB04806C9A4343
:109B500002434A6010BD0000F8B50446002680307C
:109B60000660FDF729F8054620680068124F0007D7
:109B700009D501212B46002249052046009700F017
:109B8000A1FA00280DD12068006840070BD50121FB
:109B90002B46002289052046009700F093FA002802
:109BA00001D00320F8BD2020A067E067266660345E
:109BB00026750020F8BD0000FFFFFF01F8B5154C29
:109BC000C826E078002823D16079002820D1012020
:109BD0006071114D686B0027002818D0686BC82190
:109BE000081A0FE00D48E168405C61698847E06849
:109BF000401CE060E068C82800DBE760696BC820B3
:109C0000401A761EE168814201D0002EEADC6771BD
:109C1000F8BD00005400002000000240200D00208C
:109C200070B5224CE07800283FD1207900283CD143
:109C3000012020711E4EF16900250906002933DA42
:109C40002156625791420AD1F06940062CD5A0797D
:109C5000002829D0A5712089401C208124E0A17909
:109C6000002903D1A0710A2000F08BFD00202056AE
:109C7000CC2148430F494218206912181279B26268
:109C8000401C00222061A256CC235A4389588142AD
:109C90000ADC25612078401C207020780E2800D135
:109CA0002570A078401CA070257170BD5400002064
:109CB00000380140F801002010B5806A00220146FA
:109CC00040314A834A82FDF74FFF10BD70B5846A68
:109CD000A06FE56F2168896800260906002906DA69
:109CE000212804D152200653204600F06BF820684A
:109CF0008068400606D5222D04D15A2006532046FE
:109D000000F047F8204680300168102211430160BE
:109D10002046FDF729FF70BD10B501460968806A2D
:109D2000096889061CD400225A210A5201680A686F
:109D3000FF2301339A430A6001688A68520852007F
:109D40008A6001688A6840239A438A602021C1673B
:109D5000016E012904D101680A6810239A430A6040
:109D6000016E012902D0FEF7E1F810BD5821095A11
:109D7000FDF7F8FE10BD10B5806A016E012902D012
:109D8000FEF7D5F810BD5821095A4908FDF7EAFE3B
:109D900010BD01680A68FF2321339A430A600168F5
:109DA0008A68520852008A60016E012904D1016854
:109DB0000A6810239A430A602021C16700210166C6
:109DC0004166704701680A68C0239A430A602021EF
:109DD0008167704770B5164CE278002A0CD1227961
:109DE000002A09D10122E2700025C82903DC0222E1
:109DF000A256002A01DCE57070BD0123E356CC2297
:109E000053430C4AD1500123E356CC2673439B188D
:109E10000A460146181DFBF7B1F96078401C6070D6
:109E200060780E2800D16570A078401EA070E2E72F
:109E300054000020F8010020F8B50446016880684D
:109E40002369E66918436369002533431843724A5E
:109E50000B68724E334003430B602168486803234C
:109E60001B039843E368184348602168A069914246
:109E700001D0236A18438B680B263602B343034391
:109E80008B606749236867488B420CD1C0688007A4
:109E9000800F06D0012839D0022835D0032821D1DF
:109EA0001EE001271FE060498B420AD1C0680C21E7
:109EB000084027D0042829D0082825D00C2811D103
:109EC0000EE093420ED1C16803208002014019D0F8
:109ED00001208002091A19D0091A15D0814201D136
:109EE000082700E010274F49504840398600934228
:109EF00032D1002F0CD0022F0DD0042F10D0082FFC
:109F00007FD126E00027EEE70227ECE70427EAE707
:109F1000FDF7B8FA06E00968C90605D4304603E043
:109F2000FDF7D0FA002872D06268510051188142C2
:109F300067D81103814264D3010E06025008002342
:109F400030185941FBF7EAF803210902411A384A4F
:109F500055E00120C003E7E70122E369D203934201
:109F60002BD13B0000F0E1F90906090C4D114D4DD4
:109F70004D274D00FDF786FA09E0FDF793FA06E05C
:109F80000968C90605D4304603E0FDF79BFA0028AE
:109F90003DD0616840004A088018FBF7A9F880B2FC
:109FA0000146244A103991422BD8511C0140000728
:109FB000400F084329E01046EBE73B0000F0B5F9FD
:109FC0000906090C2112212121232100FDF75AFA4B
:109FD0000AE0FDF767FA07E00968C90606D43046CB
:109FE00004E00EE0FDF76EFA002810D061684A0820
:109FF0001018FBF77DF880B201460E4A10399142E5
:10A0000003D9012503E01046F0E72168C86000206D
:10A010006066A0662846F8BD00480040F369FFEF7F
:10A0200000380140401002400044004000093D005B
:10A03000FFFC0F00EFFF0000F8B50446416540301B
:10A0400000262746028380373E602220E0672546AF
:10A05000206F603500281CD01749C162216F174856
:10A060000863216F16484863206F8663236F606D15
:10A070009C4613462168024660462431FCF7F4FBF7
:10A08000002806D0102038602E752020A0670120FF
:10A09000F8BD2E7520680168FF220132114301606E
:10A0A0002068816801221143816020688168402214
:10A0B000114381600020F8BD199D0008779D0008BC
:10A0C000CD9C0008FFB581B005460F4604466035BB
:10A0D0000A9E39E0701C37D0FCF76EFD0499401AD7
:10A0E000B04222D8002E20D02068016849072BD525
:10A0F000C069C043000527D401202168C00208625E
:10A1000020680168FF22A1329143016020688168C4
:10A110004908490081602020A067E0678034206002
:10A1200000202875032005B0F0BD20680168FF22DB
:10A13000A13291430160206881684908490081602B
:10A140002020A067E067EBE72068C16938468843B4
:10A1500005D0002103988142BCD00020E3E7012113
:10A16000F8E7000010B504491020096808620248A9
:10A17000FDF7FCFC10BD0000CC16002001490D20AD
:10A18000887070475400002010B5FEF797FAFEF76C
:10A1900077FBC82202490348FDF798FE10BD000076
:10A1A000200D0020CC160020F8B53E4C002321786D
:10A1B0003D4A1D46082910D0072947D0062950D00E
:10A1C000052952D0042953D0032954D0002956D050
:10A1D000012958D002295AD05BE0A17800264A1FF5
:10A1E00004E0314FBF5DFB189BB2761C9642F8DB52
:10A1F000667927799A195118E3786278C91889180D
:10A20000C9194018C0430006000E1AD1012E14D0FF
:10A21000022E16D125482449C018FAF7AFFF01F0E5
:10A220008DFF642000F0A6FABFF34F8F214920482C
:10A23000C860BFF34F8F00BFFDE759081046FFF716
:10A2400081FA2570E570A570A571F8BDA17950540B
:10A25000491CC8B2A071A178491F8842F5D10820D5
:10A2600001E0607007202070F8BDE0700620FAE77A
:10A2700060710520F7E7A070E5700420F3E755282A
:10A2800007D10120EFE7AA2803D10220EBE703283A
:10A2900003D02570E570A570F8BD032020702071F3
:10A2A000F8BD000034010020DE140020E80D00207D
:10A2B0000400FA0500ED00E010B5024A024900F082
:10A2C000E5F910BD75B40008880100202021020CBA
:10A2D00001D010211046020A01D0104608390209A7
:10A2E00001D01046091F820801D01046891E42087D
:10A2F00001D0881E7047081A7047F8B5040C8BB25D
:10A30000264682B25E430D0C1046370C5843360485
:10A3100080190021794116466E43370C36048019A6
:10A32000794126466E438919F8BD30B47446641EDF
:10A330002578641CAB4200D21D46635D5B00E318C8
:10A3400030BC18474900CA020243100000D0042064
:10A350004A0D01D001221043044A490D914201D116
:10A3600002210843012800D105207047FF070000A3
:10A370008307FF22DB0E9A408907090E99400028C7
:10A3800008DB830809489B001B18186890430843A2
:10A39000186070470007000F0838830804489B00C6
:10A3A0001B18D86990430843D861704700E400E067
:10A3B00000ED00E0BFF34F8F04490348C860BFF3CE
:10A3C0004F8F00BFFDE700000400FA0500ED00E03C
:10A3D000F8B504464F1EC8000838211815461E4619
:10A3E000086849683A4606239A4310D02A463346FD
:10A3F000FBF74AF83A46D200083AA3181A687F1EBB
:10A400005B68FAF78FFF06223B469343EED1022F9B
:10A4100023D0042F11D0062F2FD12A463346FBF725
:10A4200033F8E36AA26AFAF77DFF2A463346FBF760
:10A430002BF8636A226AFAF775FF2A463346FBF760
:10A4400023F8E369A269FAF76DFF2A463346FBF762
:10A450001BF863692269FAF765FF2A463346FBF762
:10A4600013F8E368A268FAF75DFF2A463346FBF764
:10A470000BF863682268FAF755FFF8BD002210B5A3
:10A48000134610460149FBF767F810BD0000F03F86
:10A4900010B5FAF747FF10BD002210B5134610465D
:10A4A0001146FBF759F810BD10B50721024A0020EC
:10A4B0000907FBF7C9F810BD01030000034A10B5F6
:10A4C00000201107FBF7C0F810BD000001FDFFFFE1
:10A4D00002E008C8121F08C1002AFAD1704770476D
:10A4E000002001E001C1121F002AFBD170470000CB
:10A4F00001490860704700008C01002008B5002168
:10A50000684601706B46012202212C2000F052FFA8
:10A510000221684601706B4601222C2000F04AFFA0
:10A5200008BD000038B504466D20694608706B46CA
:10A53000012207492E2000F03DFF0649002C01D0E2
:10A54000054A00E0054A2E2000F01AFF38BD000041
:10A5500006080000061800000706000007160000A5
:10A5600038B504466B4602220021362000F0EEFD8D
:10A57000B3212300FFF7D9FE0E0F08153A3A3A3AF5
:10A580001C273A3A2F34483A002168460170407837
:10A590004108490014E06946087880088000401CA2
:10A5A00004E06946087880088000801C08701DE07F
:10A5B000684602780A4048320270417880200143A0
:10A5C0006846417012E0684602780A40027040789E
:10A5D0004106490EF4E7694648780221084303E042
:10A5E00069464878FD210840694648706B4601225B
:10A5F0000021362000F0DEFE012200AB114636209D
:10A60000013300F0D7FE38BD69460878CF210840F5
:10A6100069462030CAE708B5032168464170012128
:10A6200001706B4602220021362000F0C3FE012299
:10A63000D20306212D2000F0A3FE012000F09AF89D
:10A640000120FFF78DFF08BD08B5020A69464A7070
:10A6500008706B46022204212D2000F0ABFE03207F
:10A66000694608706B46012206212D2000F0A2FEEB
:10A670000020694608706B46012206212D2000F05B
:10A6800099FE0A212D2000F047FD08BDF8B51646B9
:10A690000F460446002503E03946B047641C6D1C94
:10A6A00020780028F8D12846F8BD0000F8B54A0007
:10A6B0002B4B520DD6182B4A0C460546142E2BDA7E
:10A6C000002E12DA284BFAF72DFE00221346FBF774
:10A6D00083F840D2002C03DA0124E40700253AE095
:10A6E0002046284337D0214C14E0214F0B46F74039
:10A6F0003B402B4331D01C4BFAF714FE002213468B
:10A70000FBF76AF827D2002C03DD01200005F0409A
:10A710000419BC4300251EE0332E1EDC33460027FF
:10A72000143BFF43DF40384217D00F4BFAF7A4FE2B
:10A7300000221346FBF750F80DD2002C0ADD142E30
:10A740000CD03420811B012088404019A84200D23F
:10A75000641C0546BD4321462846F8BD641CF9E744
:10A7600001FCFFFF9C7500883CE4377E0000F03F51
:10A77000FFFF0F007D2110B5C900484300F001F82C
:10A7800010BD002140E000BF00BF00BF00BF00BF00
:10A7900000BF00BF00BF00BF00BF00BF00BF00BFC1
:10A7A00000BF00BF00BF00BF00BF00BF00BF00BFB1
:10A7B00000BF00BF00BF00BF00BF00BF00BF00BFA1
:10A7C00000BF00BF00BF00BF00BF00BF00BF00BF91
:10A7D00000BF00BF00BF00BF00BF00BF00BF00BF81
:10A7E00000BF00BF00BF00BF00BF00BF00BF00BF71
:10A7F00000BF00BF00BF00BF00BF00BF00BF00BF61
:10A8000000BF00BF00BF491C8142BCD37047FFB5E9
:10A8100081B01E460F46040026D00B9903980143D1
:10A82000A06A3943826807209047002818DB0A99FC
:10A83000A06A3143826806209047002810DB254635
:10A840002035A979032F01D908200143032E01D90E
:10A8500004200143A06A826809209047002806DA94
:10A860000120C04305B0F0BD0020C043FAE73846E0
:10A8700000F000F92060304600F0FCF860600A98B3
:10A8800068700398A870EF702E710B9868710020A3
:10A89000E8E70000F7B50446002090B00090019072
:10A8A000002C05D06A46062101F082FC062803DA56
:10A8B0000020C04313B0F0BD6846407801026846EE
:10A8C000007800040918684680780818FAF7F8FE3E
:10A8D000054668460391007901026846C078000485
:10A8E0000918684640790818FAF7EAFE0322064676
:10A8F0000F4692075C4BFAF76FFF07D200225B4BC3
:10A9000030463946FAF7B2FD06460F460322920753
:10A91000554B28460399FAF75FFF07D20022534BA5
:10A9200028460399FAF7A2FD054603912068FAF735
:10A93000C7FE02460B4630463946FAF70DFE07467B
:10A940000A200791205EFAF7A7FE3A46079BFAF71E
:10A950009BFD064608200991205EFAF78BFE002138
:10A96000C943FAF7D3FCFAF70FFF3246099BFAF70F
:10A97000D9FC069108906068FAF7A2FE02460B46E1
:10A9800028460399FAF7E8FD05461A200E46205E90
:10A99000FAF782FE2A463346FAF776FD0C900991C3
:10A9A0001620205EFAF778FE099B0C9AFAF7BAFC9B
:10A9B00005910A902A46334638460799FAF764FD0E
:10A9C000059B0A9AFAF760FD05910A901420205E13
:10A9D000FAF762FE3A46079BFAF756FD07461C2037
:10A9E0000791205EFAF758FE2A463346FAF74CFDE7
:10A9F0000E900B911820205EFAF74EFE0B9B0E9ADC
:10AA0000FAF790FC2A463346FAF73EFD0B910E907A
:10AA10002069FAF741FE0B9B0E9AFAF783FC2A464F
:10AA20003346FAF731FD05460E46E068FAF734FE84
:10AA30002A463346FAF776FC3A46079BFAF772FC49
:10AA4000059B0A9AFAF76EFC01229207084BFAF767
:10AA50001BFD02460B46129C0898069903C41198E8
:10AA60000CC0002026E70000FFFF5F41000070419E
:10AA7000E17A843F00B50121C9040300FFF755FCCA
:10AA8000081A05080B0E1114171A0320C00400BD84
:10AA90000720C00400BD0F20C00400BD1F204003DC
:10AAA00000BD3F20400300BD7F20400300BDFF20CC
:10AAB000400300BD084600BDFEB5264F0D4604000C
:10AAC0000FD0002D0DD0264600202036B071F07139
:10AAD00029680D208847002801DA7800FEBD10287B
:10AAE00001D03846FEBDA562E968002901D02820C2
:10AAF0008847204600F030F80028F3DBA06AA52143
:10AB000082680E209047A06A962182680F209047A5
:10AB1000A06A0221826862209047A06A00218268B0
:10AB20000E209047A06A002182680F20904771791B
:10AB30003020019100900623202201212046FFF7BA
:10AB400066FE0028CEDB204600F0AEF80028C9DB08
:10AB50000020FEBDFFFFFFFF10B586B004461421A4
:10AB60006846FAF724FB002C7ED0A06A12214368C5
:10AB70006A4610209847122877D16846007801224B
:10AB800001016846407812030009081843492081F2
:10AB9000884201DD801A208168468378407800076A
:10ABA000000D18186081884201DD801A60816846B6
:10ABB0000079012201016846C078120500030918D6
:10ABC00068464079000908183549E060884201DD8F
:10ABD000801AE060684640790007030B6846807978
:10ABE00000021B186846C07918182061884201DDF0
:10ABF000801A20616846417A007A0002081802B281
:10AC0000284801210904A282824201DD521AA2824F
:10AC10006A46D37A927A12029A1812B2E282824279
:10AC200001DD521AE2826A46537B127B12029A18A5
:10AC300012B22283824201DD521A22836A46D37BFA
:10AC4000927B12029A1812B26283824201DD521A7A
:10AC500062836A46537C127C12029A1812B2A28353
:10AC6000824204DD501A01E00BE008E0A083A06AF4
:10AC7000016828208847002806DA0120C04306B072
:10AC800010BD0020C043FAE7C011C00720340028DF
:10AC900000D0802060710020F1E70000FF07000075
:10ACA000FFFF0700FF7F000010B5040009D0A06A75
:10ACB0000721826808209047002805DA0120C04358
:10ACC00010BD0020C04310BD07202034207000209C
:10ACD00010BD0000FEB50446002001900090607990
:10ACE000734940000E5A61782578491E7148CFB2E9
:10ACF0000163042D77D0072D75D0002102912178B2
:10AD000001736C49E379012292058969002B6CD0AB
:10AD1000914381616748217A4173217A8269890769
:10AD2000890B0A4382610021042000F034FB324683
:10AD300061492E2000F024FB3846FFF7F3FB5F4EFD
:10AD40000522705D810040185D49431807212B20C2
:10AD500000F030FB5B49029801220B180B212820E0
:10AD600000F028FB705D584980000A580C2128200B
:10AD700000F011FBE079554980004018A1794900A5
:10AD8000425A0221272000F0FBFA51487E00825BE4
:10AD90000421272000F0F4FAE079002829D0A078D7
:10ADA00004282CD02820694608722022062127205A
:10ADB00000F0E6FA02AB01222621272000F0FAFA81
:10ADC000444938014018E178890042580821272079
:10ADD00000F0E1FAA17A601C627A0902114313D0F3
:10ADE00016E000E001E0012188E71143F6088161E7
:10ADF00090E764220621272000F0C2FAE0E7102045
:10AE0000694608720246D1E733490172090A417264
:10AE1000417A007A0A0202432021272000F0B0FA8A
:10AE20002E4F0C2123203A6800F0B5FAF0198288E1
:10AE30000421232000F0A4FAA07900280BD0E079A7
:10AE40002749012243180021212000F0B3FA0320F2
:10AE50000190012000902A07120F10010243607830
:10AE600000218007000B024301980005024300986F
:10AE7000400402432079C006400902436079C006BD
:10AE800002431F2000F087FAA0786178012308436D
:10AE900002040848DB030261E179490319430A43CC
:10AEA00002610021082000F076FA0020FEBD0000BB
:10AEB000E4C20008BC010020042800008CC2000885
:10AEC000240000204200002094C20008B4C2000800
:10AED000C0C20008C4C2000841100000ACC2000893
:10AEE0004400002038B50C4607498A8B00210243F4
:10AEF0002C2000F045FA684604706B4601220621BA
:10AF00002C2000F057FA38BDBC01002010B5FFF727
:10AF1000F5FA10BD10B504460421362000F0FCF807
:10AF20000121C902002C01D0084300E088430246F9
:10AF30000421362000F02FFA10BD000038B5402063
:10AF40006946087000210E2000F0E6F80446002251
:10AF500011460E2000F01FFA6B46012200210D2041
:10AF600000F028FA074A00210F2000F014FA00F040
:10AF7000EDF9224600210E2000F00DFA02480021D2
:10AF8000017338BDF8FF2724DC010020FEB505461B
:10AF9000042069460870514C00206075214620311C
:10AFA000206348710873A0836063A06300F0C8F851
:10AFB0004B4E206002E000F0C3F82060B042FAD1AE
:10AFC0000020FFF7CDFA00F0BBF8464E2060307845
:10AFD000242801D9243806E00621FAF789F8062248
:10AFE000101A40010843020601040A4301020A4301
:10AFF0000243B260706000211E2000F0CCF900F026
:10B000009FF820606B4601220021242000F0D2F935
:10B010001E20FFF719FB86B2300AA0730420FFF749
:10B0200013FB074600F08CF820603806000E0DD0A8
:10B0300002206946087101AB012212212D2000F087
:10B04000B9F9A08B012109030843A08300F078F827
:10B0500020600620FFF7F8FA60600720FFF7F4FA97
:10B06000A060F006C00E207501D110202075C0B27E
:10B0700000F0DCF9E80707D0FFF7CDFAA08B01213B
:10B08000C9020843A0830AE00521362000F02EF80B
:10B090001549084002460521362000F071F90120CB
:10B0A000FFF75EFA0021042000F036F8A0610021CD
:10B0B000262000F031F815218903084302460021BB
:10B0C000262000F068F900222621362000F058F9E9
:10B0D00000F036F820600020FEBD0000BC0100201A
:10B0E0003001CADE18000020FFFD000038B5094C11
:10B0F00089B280B26B46022200F028F8002806D1FF
:10B1000068464078010268460078081884B22046F4
:10B1100038BD0000FFFF000038B50024E44389B2C9
:10B1200080B26B46042200F011F8002806D10321FA
:10B130006846435C2202D418491EFAD5204638BD21
:10B1400010B500210846FFF7E7FF10BD38B500290C
:10B1500009D0402420436C462070C8B27F2906D80D
:10B16000607002200AE069460870012006E0802431
:10B1700020436C466070C809A0700320694600F047
:10B18000B7FF38BD10B5144603460A4621461120C4
:10B19000FFF7DCFF10BD10B5034605220021152086
:10B1A000FFF7D4FF10BD10B503460522002117207C
:10B1B000FFF7CCFF10BD38B5054600206946087082
:10B1C00000F0C4F8FF2401342246002D01D00322F0
:10B1D000120200210D2000F0D3F8002D13D06B4691
:10B1E000012203210F20FFF7B1FF68460078000716
:10B1F00009D5FFF7A3FE224600210D2000F0C0F87C
:10B200000020C04338BD002038BD10B502460121E2
:10B210000A2000F0C0F810BD10B5044600211A2025
:10B22000FFF77AFF000D22030005120B02430021F5
:10B230001A2000F0B0F810BD10B5024602492E20C9
:10B2400000F09EF810BD000004180000F8B5054697
:10B250006B46012203210420FFF778FF0126114CE1
:10B260003607002D0DD02A4600210C2000F088F86A
:10B27000694608781021084369460870A069304380
:10B2800007E069460878EF21084069460870A06920
:10B29000B0430B46A06101220321042000F08AF88C
:10B2A000F8BD0000BC01002010B5024600211820A6
:10B2B00000F066F810BD0000F8B5074600256846A6
:10B2C0000570B807204C2E4600280ADA802069460F
:10B2D00008706B46012200210D2000F06BF8012060
:10B2E0002073F8076946087821D00621084369468B
:10B2F00008706B46012200210D2000F05BF803214D
:10B300000F20FFF7F3FE8121C900084219D0402029
:10B31000694608706B46012200210D2000F04AF8B2
:10B320000020FFF7F7FD00252673ED4309E0022119
:10B330000843694608706B46012200210D2000F089
:10B3400039F82846F8BD0000DC0100201CB56B462A
:10B35000012203210F20FFF7F9FE68460078402202
:10B36000C1091040C9014000814208D0012069464E
:10B370000871024601AB03210D2000F01BF81CBD33
:10B3800008B56B461A70120A5A7089B280B202224E
:10B3900000F010F808BD38B500236C46E254120ADC
:10B3A0005B1C042BFADB89B280B22346042200F036
:10B3B00001F838BD38B58024002909D0C0252843BC
:10B3C0006D462870C8B27F2907D86870022009E04E
:10B3D000204369460870012004E020436870C809D2
:10B3E000A8700320694600F02DFF38BD10B5144643
:10B3F000012312189B029A4202D90020C04310BDBB
:10B400000B46821E21460920FFF7D4FF002010BD05
:10B4100010B5054A8905126901430A430021082035
:10B42000FFF7B9FF002010BDBC01002038B504466D
:10B430006B4601220E212B20FFF788FE684600781C
:10B44000E10640094001C90E0143684601706B46A0
:10B4500001220E212B20FFF7ADFF38BD10B50021D2
:10B4600042541C06120A22431B0A491C0429F7DB1A
:10B4700010BD000013B501231A4669460248FCF7C7
:10B4800057FD00981CBD0000CC1600207CB50024A0
:10B4900025466846FFF77FFE04206946220E2D02EE
:10B4A000154322020C5C1443401EF7D52046294662
:10B4B0007CBD7CB5002425466846FFF774FE042059
:10B4C0006946220E2D02154322020C5C1443401ED5
:10B4D000F7D5204629467CBDFBF77CFBFEF7D2F969
:10B4E000FDF700F941494248002522C00560856109
:10B4F000C56140490562C1600838FBF7FDFCFDF7F6
:10B50000DDF8FDF7BDF9FDF799F9FDF7A3F8012185
:10B51000002289023848FBF748FB05240122240752
:10B52000D1032046FBF741FBFDF752FFFCF77AFF02
:10B53000FAF734FBFAF7B6FBFAF784FBFCF77AFD6F
:10B540000721A015FFF7CEFCFFF7E0FC0122110355
:10B550002046FBF72AFB2648C8222849C830FCF7BA
:10B56000B5FC274F274E284C387800280FD130786B
:10B57000002801D003280AD10121C9021E48FBF787
:10B5800007FB002803D101210846FBF7C9FDE0783D
:10B59000002828D06078002825D0E57072B6207881
:10B5A0000F280AD90120144900038861FEF7EEF93B
:10B5B00001201149000388620CE0012251030E486A
:10B5C000FBF7F3FAFEF7E2F90121002249030A48EA
:10B5D000FBF7EBFA62B6FCF74BFE208C0028C3D0D9
:10B5E000401E2084C0E7FCF743FEBDE7007C00401E
:10B5F00004160020FFFF000000040050200D002072
:10B600005A000020840000203C01002010B586B0C4
:10B610001748FBF7F4FB14216846F9F7C8FD1548F5
:10B620000090032001900020029005206946000749
:10B63000FBF7F2F969461048FBF7EEF969460F4847
:10B64000FBF7EAF901210846FBF76AFDFF24013404
:10B650002046FBF73DFD0A490868042210430860B4
:10B660002046FBF745FDFBF74BFD06B010BD000083
:10B6700004160020FFFF00000004005000080050E6
:10B680000070004010B50122920217491748FAF7DE
:10B690008BFB1548164902888A4223D00180042179
:10B6A0008180FF21F531C1800A21018100211E2204
:10B6B0004181D24382810122C28181834323C38697
:10B6C00002230387782343878287C287024640325A
:10B6D000118451849184C1839180142383821182C7
:10B6E00000F02CFD10BD0000E80D002000FC00085B
:10B6F000AA550000F0B51FB496B084460C46024629
:10B70000199D189803904900680063004908400893
:10B710000193002A01D0012600E000269E19FE4B6D
:10B72000F6185B109E422BD36E00039F0296002FEB
:10B7300000D00127F719F84EF84BBE199E421FD3CF
:10B74000039E0346F64F334309D03B469C4201D14A
:10B75000002A04D0019B002A05D0012604E0002025
:10B7600039461BB0F0BD00269E19EE4B9E4207D80D
:10B77000039F029E002F00D00127F6199E4207D991
:10B780002B4660462146189AFEF782FE1BB0F0BD9C
:10B790000023002C29DAE44EB04226DAE34EB04210
:10B7A00001DB022321E0DE4EB0421EDBE04E070D3E
:10B7B000BE19142E09DD3427BF1B039EFE400196DF
:10B7C000BE40039FBE420BD00FE0039F002F0CD161
:10B7D0001427BF1B0646FE400196BE40864204D198
:10B7E000019BDE07F60F02239B1B0E46164318D162
:10B7F000002D16DA002C03D0022B01D0012B06D02D
:10B800000220FEF775FEFEF739FE1BB0F0BD0220E8
:10B81000FEF76EFEFEF732FE0122D20751401BB04A
:10B82000F0BD039E002E61D1BF4EB04220D1C14871
:10B83000844201D1002A08D0B948814209DB002D99
:10B8400010DB189829461BB0F0BD0020B4491BB08E
:10B85000F0BD002D06DA01222946D2071898514082
:10B860001BB0F0BDB4497944086849681BB0F0BD0D
:10B87000AB4FB84225D1002D1FDA002904D0B142C8
:10B8800012D1002A09D018E0002A72D1A649E20F8D
:10B890000020D20711431BB0F0BD0020E20F01468B
:10B8A000D20711431BB0F0BDB14206DA2346002097
:10B8B0003946F9F751FE1BB0F0BD104621461BB0CA
:10B8C000F0BDB14212DA0126B607B54203D12346D4
:10B8D00010461946FEE3994EB54207D1261E05DBF8
:10B8E0001046314600F040FC1BB0F0BD67007F08F9
:10B8F0001646002A40D100290AD08B4A914229D10C
:10B90000002C0EDD002D1CDB002011461BB0F0BD0D
:10B91000022B16D0002C14D0012B12D1002C14DBDA
:10B920000FE0002C28DA002D09DB012B03D00020CA
:10B930007D491BB0F0BD002081491BB0F0BD012B3B
:10B9400003D0002001461BB0F0BD00200121C90733
:10B950001BB0F0BD724A91420ED1002C01DA002BCF
:10B9600017D0022B06D00020C043F9F795FE1BB07C
:10B97000F0BD90E20120F8E7E217521C94461A430A
:10B9800007D000220892664C62465B1E1A4307D01D
:10B9900009E00120FEF7ACFDFEF77EFD1BB0F0BD17
:10B9A0000022644C0892674A90427DDD664B674AEC
:10B9B00098421FDD914202DC002D05DB4DE0584826
:10B9C000814217DB002D48DD0220FEF791FDFEF7D6
:10B9D0006BFD05460E460022534B21460898F9F7A9
:10B9E00053FD084671004908C00FC00701432846AF
:10B9F0001BB0F0BD914215DA002D2EDA0220FEF7C1
:10BA000077FDFEF751FD05460E460022464B2146C6
:10BA10000898F9F739FD72005208C80FC0070243B1
:10BA2000114617E03E4B994223DD002D15DD022023
:10BA3000FEF75EFDFEF738FD05460E4600223A4B46
:10BA400021460898F9F720FD084671004908C00F03
:10BA5000C007014328461BB0F0BD0220FEF748FD99
:10BA6000FEF72CFD49004908E20FD20711431BB035
:10BA7000F0BD002230463946F9F7F8FC01220546B0
:10BA80000E46D243F9F7E0FD314A324BF9F7F4FCA8
:10BA90002A463346F9F7F8FC0022284BF9F7ECFC6C
:10BAA00007462A46334600E064E0039110461946F3
:10BAB000F9F7EAFC3A46039BF9F7E6FC074603224E
:10BAC00009915207244B28463146F9F7DDFC0791CE
:10BAD0000C90224A204B38460999F9F7D5FC0746C5
:10BAE00001911F4A1F4B28463146F9F7CDFC3A46D3
:10BAF000019BF9F7BBFC07460B46024609910799E3
:10BB00000C98F9F70FFC00250E462846079B0C9A67
:10BB1000F9F7ACFC3A4627E0FFFF1F00FFFF0F00DC
:10BB20000000F03F0000E0FF0000F07F0000404315
:10BB300001FCFFFF0000F0BF560B00000000E03FDB
:10BB40000000F0FF0000E0410000F043FFFFEF3F86
:10BB5000555555555555D53F4715F73FFE822B6531
:10BB600044DF5DF80BAE543E099BF9F785FC0246B5
:10BB70000B4652E1012500202D05A94207DA3522A6
:10BB800030463946F9F760FD06463420C0430A15B1
:10BB90001218FE48101803900803FD49000B0143DA
:10BBA0000F46FC49884201DC002003E0FA49884244
:10BBB00002DA0120119005E0002011900398401C4A
:10BBC0007F1B039011980597C200F4480F927844A8
:10BBD000801843680268394630460D930292F9F79F
:10BBE00045FC07910C9030460D9B029A0599F9F798
:10BBF00099FB02460B460020E549F9F7ADFC099197
:10BC00000490079B0C9AF9F73FFC129000201090CB
:10BC1000E3480D46784400680E90012178104907EA
:10BC2000084311990D9B890440180121C904471844
:10BC30003946029A0E98F9F719FC3246059BF9F736
:10BC40001BFC02460B4629461098F9F71DFC0646D8
:10BC500002913B4629460E9A1098F9F715FC079B6E
:10BC60000C9AF9F709FC3246029BF9F7FFFB099B96
:10BC7000049AF9F709FC0591129A0A902B4610468E
:10BC80001946F9F701FC06460246C6480F460B4620
:10BC900006217844FEF79CFB32463B460091049017
:10BCA00010461946F9F7F0FB009B049AF9F7ECFBF4
:10BCB00006460F462B461946129A1098F9F732FBA2
:10BCC000059B0A9AF9F7E0FB32463B46F9F72AFB57
:10BCD000109A079104902B4610461946F9F7D4FBA9
:10BCE000B14E0022334609910290F9F71BFB079BE6
:10BCF000049AF9F717FB00200746024633460091E5
:10BD0000F9F7B4FB099B029AF9F7B0FB079B049A79
:10BD1000F9F7B2FB06460D913A462946009B10986A
:10BD2000F9F7B2FB07910C902B463046129A0D9909
:10BD3000F9F7AAFB05460E463A46009B05990A9874
:10BD4000F9F7A2FB33462A46F9F7ECFA02460B460E
:10BD50000746099107990C98F9F7E4FA00250E4671
:10BD60002846079B0C9AF9F781FB3A46099BF9F79D
:10BD700083FB07460722099152078C4B3146284620
:10BD8000F9F782FB07910090894A884B3846099958
:10BD9000F9F77AFB07460191864A874B31462846D8
:10BDA000F9F772FB3A46019BF9F7BCFA834B7B44E7
:10BDB0000F9A9B181A685B68F9F7B4FA0290099118
:10BDC0000398F9F769FC05910490099B029A079979
:10BDD0000098F9F7A7FA7A4B7B440F9A9B181A68D8
:10BDE0005B6817460393F9F79DFA059B049AF9F7E8
:10BDF00099FA0E462846059B049AF9F737FB3A460E
:10BE0000039BF9F733FB079B009AF9F72FFB099B7C
:10BE1000029AF9F731FB02460B46199900200C9063
:10BE20000F461898F9F730FB029104903B460C9AA4
:10BE300019991898F9F71AFB2A463346F9F724FBA3
:10BE4000029B049AF9F76EFA09910E902A4633463E
:10BE500039460C98F9F718FB06460F46099B0E9ACF
:10BE6000F9F760FA574A0D46914220DB5242AA1870
:10BE7000024310D132463B46F9F7F8FA0490039199
:10BE8000514A524B09990E98F9F74CFA039B049AC0
:10BE9000F9F7A2FC1ED20220FEF72AFBFEF704FBF4
:10BEA00049004908E20FD20711431BB0F0BD6A00F8
:10BEB000474B52089A420DD3464AAA18024300D073
:10BEC000CBE532463B46F9F7D1FA099B0E9AF9F7D2
:10BED00083FCF5D96800002340082C490393020D28
:10BEE0003D4B5218984223DD01200005521CD040E2
:10BEF00042195000400D40183849794409681346EA
:10BF00008C463749C1408B4312030121120B0905AE
:10BF100051181422101AC1400391002D01DA484231
:10BF20000390624630463946F9F7A0FA06460F46B6
:10BF300032463B4609990E98F9F7F4F900252A464E
:10BF4000284B28460591F9F79FFA07910C90264A4D
:10BF5000264B28460599F9F797FA00910290324648
:10BF60003B4628460599F9F781FA099B0E9AF9F79D
:10BF700083FA1F4A1F4BF9F787FA009B029AF9F7D9
:10BF8000D1F907460B460246099135E001FCFFFF57
:10BF90000000F03F8E9803007AB60B0066070000A1
:10BFA000A8070000D20600000000084009C7EE3FC5
:10BFB000FD033ADCF5015B14E02F3EBEA605000050
:10BFC0006C05000000009040FE822B654715973CF1
:10BFD00000CC904000346F3F0000E03FC2040000FE
:10BFE000FFFF0F00432EE63F396CA80C615C20BEBA
:10BFF000EF39FAFE422EE63F07990C98F9F792F9CD
:10C0000005460E46079B0C9AF9F730FA3A46099B0B
:10C01000F9F732FA09912A4633460E90104619462E
:10C02000F9F732FA074602462F480B4605910521DB
:10C030007844FEF7CDF93A46059BF9F725FA2A46EA
:10C040003346F9F719FA0746019128463146099B0C
:10C050000E9AF9F719FA099B0E9AF9F763F9012379
:10C0600004910C9000229B0738460199F9F7FEF9DC
:10C0700005910E903A4628463146019BF9F704FA9D
:10C08000059B0E9AF9F768FA049B0C9AF9F7EEF9FA
:10C090002A463346F9F7EAF90022144BF9F7ECF98E
:10C0A000064603980D46000541190915002912DCC2
:10C0B00030462946039AF9F7C7FAFEF743F90428F0
:10C0C00001D1FEF7FBF930462946039AF9F7BCFA8D
:10C0D000064601E004E029180B463246214608983E
:10C0E000F9F7D2F91BB0F0BD640300000000F03F87
:10C0F000F0B58C4600251026052109078E620E4CEE
:10C1000008E067467F5DE760A768FF07FCD0E76847
:10C110001F706D1C8542F4DB0020074606E0E760D7
:10C12000A568ED07FCD0E5681D54401C9042F6D38D
:10C130008E610020F0BD00000030014070B572B685
:10C140000124074DA40221462846F9F713FE0028D2
:10C1500004D0224603492846F9F7B0FE62B670BD06
:10C1600000FC0008E80D0020F8B506460C46F9F77B
:10C1700041FC051E0F4600D00120014349000B4839
:10C180004908411AC90F0DD0002E01D0012100E04D
:10C1900000210C4361004908401AC00F02D1012060
:10C1A000FEF7A6F928463946F8BD00000000F07FEA
:10C1B000F8B515460E460746002407E03819C0B208
:10C1C00000F008F8641C2870E4B26D1CB442F5D38A
:10C1D0003046F8BD10B50446FBF7E6FFEE20FBF74E
:10C1E000B6FFFCF71AF82046FBF7B1FFFCF715F88D
:10C1F000FBF7DAFFEF20FBF7AAFFFCF70EF80020B1
:10C20000FBF778FF0446FBF7EAFF204610BD7047B6
:10C2100070B50D460446FBF7C7FFEE20FBF797FF0E
:10C22000FBF7FBFF2046FBF792FFFBF7F6FF2846E4
:10C23000FBF78DFFFBF7F1FFFBF7D1FF0A20FEF7BD
:10C24000A0FA70BDF0B50025102605279C463F07D3
:10C250000B46BE620C4C06E0595DE160A168C9075F
:10C26000FCD0E1686D1C8542F6DB002007E06146EA
:10C27000095CE160A168C907FCD0E168401C9042FC
:10C28000F5D3BE610020F0BD003001400000010286
:10C2900003040005405C0000A05C0400C06C0800C2
:10C2A000805C0400E03F1E00E07D1E0007A902251F
:10C2B00070889B880A001600010006000100020039
:10C2C00087008D002D001A3152001A339A001A355A
:10C2D0001D011A376B003B31BE003B335E013B351D
:10C2E00096023B37000099599959EB518F421E45F0
:10C2F000142E0080EB51F5283333E13A703DE13ADA
:10C30000C235852BC2353333C235C235AE47E13A2B
:10C310005138A33051380000000000000000010235
:10C32000030406070809030406080C10182030004F
:10C330000000000102030400000000000000F03FC4
:10C34000000000000000F83F0000000000000000B6
:10C350000000004003B8E23F0000000000000000C1
:10C3600006D0CF43EBFD4C3E033333333333E33F4F
:10C37000FFAB6FDBB66DDB3F4D268F515555D53F7B
:10C3800001411DA96074D13F65DBC9934A86CD3F49
:10C39000EF4E454A287ECA3F3E5555555555C53F37
:10C3A00093BDBE166CC166BF2CDE25AF6A56113F29
:10C3B000F16BD2C541BDBBBED0A4BE726937663E2B
:10C3C0000000000000000000E8C30008000000209A
:10C3D00090010000BC5A00084CC4000890010020E5
:10C3E000681A0000E0A400080124130704380D09AE
:10C3F0001E080540082609104008560A131D043B74
:10C4000008BE0516D8BC4010085201033CC84207BC
:10C410006E52030CE5800C1B0202DD14090102229E
:10C4200081F01F6681049889968696798215980313
:10C43000981498879674977882439788967197771F
:0CC440008249F10139293F92049220004A
:04000005080050C1DE
:00000001FF
